:020000040000FA
:06000000CCEF34F0120009
:0600080080EF2EF0120053
:06002A000600306A000030
:1000300075030000040000000E6A00009602000034
:1000400022000000E66900006E02000028000000A7
:10005000E4690000FD01000002000000E269000008
:10006000FE00000002000000D26900002D03000025
:04007000100000007C
:0C0074000901006B0A0E005D26E200513D
:10008000220DF3CF01F9F4CF02F9000E01270A0E79
:100090000223DFEC08F0EF6A34EC0AF0EF9034EC66
:1000A0000AF0EF8234EC0AF0EF8434EC0AF0EF98B7
:1000B00034EC0AF0EF96DFEC08F0EFEC09F0DFEC3F
:1000C00008F003EC0AF0002BD7D70101496B040EAE
:1000D0004A6F4B6B4C6B4D6B4E6B12000901006B02
:1000E0000A0E005D36E20051220DF3CF01F9F4CF84
:1000F00002F9000E01270A0E0223CEEC08F0EF50A1
:10010000000925E1CEEC08F0010EEF6ECEEC08F010
:100110000B0E4FC1EBFF0C0E50C1EBFFCEEC08F005
:100120000D0EEB6A0E0EEB6ACEEC08F0FFEC09F058
:1001300046EC0AF0EF8046EC0AF0EF96CEEC08F0C1
:10014000EFEC09F046EC0AF0EF8200511200002BB0
:10015000C7D7FE0C09016F6B6C6B0A0E6C5D14E265
:100160006C51220DF3CF6DF9F4CF6EF9000E6D27AF
:100170000A0E6E2385EC08F0EF50000903E1010E32
:100180006F6F02D06C2BE9D76F5101E1FE0C0101BA
:10019000492B000E4A2385EC08F00B0E49C1EBFFFA
:1001A0000C0E4AC1EBFF880ED8804955130E4A55F4
:1001B00003E2496B040E4A6F85EC08F0A1EC09F0EC
:1001C000EF9085EC08F00D0E53C1EBFF0E0E54C1FD
:1001D000EBFF4B2B000E4C234D234E2307EC0AF074
:1001E00043EC09F085EC08F0180E6DEC08F067ECB4
:1001F00009F00A0EE66EE66A51C1E6FF52C1E6FF5B
:1002000085EC08F08FEC08F0F9EC08F00101020E23
:100210007E6F85EC08F0F3EC09F007EC0AF0E9ECEE
:1002200008F085EC08F0F7EC09F085EC08F0FBEC41
:1002300009F085EC08F0D8EC08F085EC08F0030E26
:10024000EF6E07EC0AF093EC09F085EC08F0F2ECA5
:1002500008F009016C51120001015551A8EC08F099
:10026000EF50040801E0000C010C01015651220D71
:10027000F3CF81F9F4CF82F9000E090181270A0E2C
:100280008223E4EC08F0EF50040806E081C988F10D
:1002900082C989F1CCEF06F056C160F14CD9F9EC76
:1002A00008F00101110E7E6FE4EC08F0F3EC09F0A8
:1002B000E4EC08F037EC0AF0E9EC08F0E4EC08F0C4
:1002C000F7EC09F0E4EC08F0FBEC09F0E4EC08F0E2
:1002D000D8EC08F0E4EC08F037EC0AF093EC09F005
:1002E000E4EC08F0050EEF6E120001015751220DEB
:1002F000F3CF83F9F4CF84F9000E090183270A0EA6
:1003000084238AEC08F09DEC09F001E1000C8AECF2
:1003100008F023EC0AF0020B01E1000C8AEC08F073
:10032000100E6DEC08F0EECF80F1EDCF81F18AEC8C
:1003300008F00F0EEB5001017F6F0101100E7E6F70
:10034000F3EC09F08AEC08F037EC0AF0E9EC08F07D
:100350008AEC08F0F7EC09F08AEC08F0FBEC09F005
:100360008AEC08F0D8EC08F08AEC08F0100EC8EC23
:1003700009F0126A136A8AEC08F037EC0AF01050A0
:10038000EE261150EE221250EE221350EE2255ECC2
:100390000AF0EF9255EC0AF0EF988AEC08F022ECA4
:1003A00009F08AEC08F0EFEC09F055EC0AF0EF8266
:1003B000010C0A0E0101585D13E25851A8EC08F037
:1003C0000F0E6DEC08F0EF50FF0802E134EF14F06F
:1003D0005851A8EC08F023EC0AF0020B02E0010CE3
:1003E000000E120001015951220DF3CF81F9F4CF13
:1003F00082F9000E090181270A0E8223D3EC08F04E
:100400009DEC09F014E1D3EC08F00F0E1BC0EBFFDC
:10041000D3EC08F0EB500201596F6CEC15F0D3EC03
:1004200008F04CEC09F0D3EC08F07BEC09F0D3ECCD
:1004300008F026EC0AF001E3000CD3EC08F0A1EC84
:1004400009F0EF885AC150F242EC14F0D3EC08F0F6
:10045000100E6DEC08F0EE2AEF22D3EC08F026EC3B
:100460000AF003E359C157F140DF010C01015B5170
:10047000220DF3CF6CF9F4CF6DF9000E09016C2752
:100480000A0E6D23B7EC08F09DEC09F014E1B7EC0F
:1004900008F00F0E1BC0EBFFB7EC08F0EB500201A9
:1004A000596F6CEC15F0B7EC08F04CEC09F0B7ECB8
:1004B00008F07BEC09F0B7EC08F026EC0AF001E359
:1004C000000C0DEC0AF0EE24106E5F51EE20116E60
:1004D000CA0ED8801054030E11540EE2B7EC08F087
:1004E000100E6DEC08F0EECF5EF1EFCF5FF1CA0EAB
:1004F000D8805E57030E5F57B7EC08F0A1EC09F007
:10050000EF885EC153F25FC154F25CC151F25DC12C
:1005100052F264EC14F00DEC0AF0EE265F51ED227D
:10052000B7EC08F026EC0AF003E35BC157F1DDDE1F
:1005300001015E51120001016051220DF3CF00F95B
:10054000F4CF01F9000E090100270A0E012300C9AA
:10055000E9FF01C9EAFF52EC0AF001E1000C7AEC74
:1005600015F000C9E9FF01C9EAFFA1EC09F0EF9617
:10057000010C01016151220DF3CF20F9F4CF21F9D3
:10058000000E090120270A0E212318EC09F052EC75
:100590000AF02BE018EC09F023EC0AF0040B08E059
:1005A000280E1DEC09F018EC09F0A1EC09F0EF940D
:1005B00018EC09F04CEC0AF0EE50ED1008E17AEC82
:1005C00015F018EC09F0A1EC09F0EF96000C18EC0E
:1005D00009F04CEC0AF0EE06EF5AE2EC14F062C1BE
:1005E000E9FF63C1EAFFEF6E010C000C01016451E9
:1005F000220DF3CF02F9F4CF03F9000E090102270F
:100600000A0E0323FFEC08F052EC0AF03AE0FFEC8C
:1006100008F023EC0AF0040B08E0280E1DEC09F0AA
:10062000FFEC08F0A1EC09F0EF94FFEC08F0120EDB
:10063000C8EC09F001016751105C6851115808E2DB
:10064000FFEC08F04CEC0AF0EECF67F1EDCF68F16B
:10065000FFEC08F04CEC0AF0EE50ED1008E17AECFB
:1006600015F0FFEC08F0A1EC09F0EF960AD067C195
:1006700057F268C158F265C155F266C156F220EFD3
:1006800015F0F36AF46A12000A0E0101695D07E2CF
:100690006951A8EC08F052EC0AF002E0010C000EDF
:1006A00012000901736B6C6B0A0E6C5D01E3D4D010
:1006B0006C51220DF3CF6DF9F4CF6EF9000E6D275A
:1006C0000A0E6E237BEC08F052EC0AF001E0C1D078
:1006D0007BEC08F023EC0AF0100B01E0BAD07BECC5
:1006E00008F0EF50000901E1B4D07BEC08F0EF50C6
:1006F000010807E17BEC08F023EC0AF0010B01E0B4
:10070000A8D07BEC08F01D0E6DEC08F00301EE5054
:10071000645D106EEE506559116E7BEC08F01F0E93
:100720006DEC08F071EC09F01050125C1150135888
:1007300001E38FD034EC14F0000901E112007BECEE
:1007400008F0F2EC08F07BEC08F01F0E6DEC08F0FE
:10075000EE2AEF227BEC08F01C0E6DEC08F0EF2A7D
:100760007BEC08F0EF50060A27E0010A25E0020AB8
:100770001CE00F0A1AE00E0A10E0060A05E0010A62
:1007800028E10901020E24D013EC0AF0106E030ECA
:10079000105C16E20901120E1BD00901110E736FD5
:1007A0007BEC08F0050EEF6E14D013EC0AF0030892
:1007B00007E30901010E0CD013EC0AF0030806E26E
:1007C0006DC988F16EC989F1E7DA03D00901100E0D
:1007D000736F0901735100083CE2100E735D11E064
:1007E0007BEC08F037EC0AF0EFCF6FF9EE2AEFCF91
:1007F00070F9EE22EFCF71F9EE22EFCF72F9EF220E
:100800000CD07BEC08F037EC0AF0EECF6FF9EECFAE
:1008100070F9EECF71F9EFCF72F9F9EC08F073C906
:100820007EF17BEC08F0F3EC09F06FC976F170C94A
:1008300077F171C978F172C979F17BEC08F0F7ECC6
:1008400009F07BEC08F0FBEC09F07BEC08F0D8EC4D
:1008500008F009016C2B28D71200140E0201576F03
:10086000586B02016C0E556F090E566F20EC15F097
:1008700001016C0E866F090E876F59DA6AC1E9FFB4
:100880006BC1EAFF4FEC0AF0EECF80F9EECF81F9B1
:10089000EECF82F9EFCF83F998EC09F0EFCF84F92E
:1008A000010E6DEC08F0EFCF85F998EC09F0020E1F
:1008B0006DEC08F0EFCF86F998EC09F0030E6DECC3
:1008C00008F0EFCF87F90901886B060E896F6EC1BA
:1008D0008AF96FC18BF96EC1D8F26FC1D9F274EC8D
:1008E00024F0F3CF8AF9F4CF8BF90C0E0201E06FFC
:1008F000E16B0201800EDE6F090EDF6FA8EC24F0C1
:10090000F3CF8DF9F4CF8EF909018D1F8E1F240EC0
:100910001DEC09F08DC950F242EC14F08EC950F272
:1009200042EC14F0140E1DEC09F06EC1E2F26FC13E
:10093000E3F204EC25F0F3CF8DF9F4CF8EF9090141
:100940007C51F31802E17D518E1903E07AEC15F029
:10095000010C55EC09F0106E116A140E105E000EB9
:10096000115A10C08FF91050106E116AE850010131
:100970006E5D6E6F11506F596F6F140E6E5F000ECB
:100980006F5B090155EC09F00201696F6A6B140E87
:100990006927000E6A2317EC17F06AC184F16BC156
:1009A00085F101016C0E826F090E836F3ED909013A
:1009B0008C6FFE0E8C5D11E26EC18FF16FC190F1F4
:1009C00001016C0E8D6F090E8E6F6AC18BF16BC1C8
:1009D0008CF18CC98AF106DA010C7AEC15F0FF0E65
:1009E00009018C5D37E101016E5109017427010194
:1009F0006F5109017523000E762377237951020B7D
:100A000003E17951010B05E0742B000E7523762369
:100A10007723EFDB0101040E7E6F70C97AF171C993
:100A20007BF172C97CF173C97DF174C976F175C926
:100A300077F176C978F177C979F16CC974F16DC92C
:100A400075F16EC972F16FC973F16AC170F16BC152
:100A500071F101D8010C72C148F973C149F974C12F
:100A60004AF975C14BF976C14CF977C14DF978C196
:100A70004EF979C14FF97AC150F97BC151F97CC166
:100A800052F97DC153F909015491549354955497E7
:100A90007EC155F98DEC15F0F3CF56F9F4CF57F927
:100AA0000901000EF35C040EF45804E3566B040EC7
:100AB000576F0DD0360ED8805655000E575505E2AB
:100AC000360E565F000E575B02D0566B576B586B55
:100AD000596B5A6B5B6B0101480E866F090E876F6D
:100AE00026D9140E01018027000E81237EA30ED08B
:100AF000040E8027000E81230901020E5C6F040E94
:100B00005D6F5E6F5F6B5499548B03D009015489FC
:100B1000549B548D549FB8C260F9B9C261F9BAC2EE
:100B200062F9BBC263F970C1E9FF71C1EAFF4FEC22
:100B30000AF0EECF64F9EECF65F9EECF66F9EFCFAC
:100B400067F9686B060E696F80C16AF981C16BF93C
:100B500080C1D8F281C1D9F274EC24F0F3CF6AF9E4
:100B6000F4CF6BF90C0E0201E06FE16B0201600E35
:100B7000DE6F090EDF6FA8EC24F0F3CF58F9F4CF45
:100B800059F90901581F591F58C946F959C947F958
:100B9000FF0E01017F5D02E11BC07FF1140E41DBFE
:100BA00080C157F381C158F30301060E566F70C11F
:100BB00054F371C155F3DFEC26F0140E0201536FAC
:100BC000546B0201480E516F090E526F64EC14F021
:100BD00001017EA30BD0040E0201536F546B02017E
:100BE0005C0E516F090E526F64EC14F0140E19DB99
:100BF00080C1E2F281C1E3F204EC25F0F3CF46F9C3
:100C0000F4CF47F9240E0DDB47C950F242EC14F043
:100C100046C950F242EC14F002016C6B6D6B7FC15F
:100C20006BF22AEC17F0C9EF16F00901FE0E036F04
:100C3000026B0A0E025D4AE202511BDB84DAEF50BE
:100C4000000941E080DA0B0EA3DB50DB020E45DA2F
:100C500048DB00011250101836E11350111833E12F
:100C600072DAEF50010802E102C903F96CDA0D0EE5
:100C70008FDB3CDB36DB1250101825E113501118C6
:100C800022E184C1E9FF85C1EAFF4FEC0AF0EECF13
:100C900014F0EECF15F0EECF16F0EFCF17F053DAD9
:100CA000EE524FEC0AF0EE5014180DE1EE5015180C
:100CB0000AE1EE50161807E1EE50171804E103E1BF
:100CC0000901025112000901022BB3D70351D1DAF5
:100CD000FE0E035D27E037DAEF50010823E10A0E2C
:100CE000E66EE66A84C1E6FF85C1E6FF2CDA17DA14
:100CF0001250FCDA020E4CDB26DA0B0E10C0EBFFB2
:100D00000C0E11C0EBFFF2DA2DDA1DDAFADA1BDA7B
:100D100018DBEF9618DA63DB16DA13DBEF820901D2
:100D200003511200FE0E035D01E1FF0CFE0CDED943
:100D3000EFCF07F9A2DBE552E750EF6ED7D92BDBF7
:100D4000020E35DB020E09DB020E2BDB020EA1DBED
:100D5000040E09DB040E30DB080E05DB080E2CDB6D
:100D60000E0E25DB0E0EF9DA0E0E1BDB0E0E91DBDE
:100D7000100E1DDB100EF1DA100E13DB100E89DBE6
:100D8000120E15DB120EE9DA120E0BDB85DB010EFB
:100D9000A4D907C9EFFF1200D1D9CFDA06E0CED926
:100DA00051DACCD91CDB84DBEF82C8D928DBC6D969
:100DB0000D0EEB6A0E0EEB6AC1D974DB02E07AEC21
:100DC00015F076DBEF96BAD91EDB72DBEF98B6D959
:100DD0003ADB010B04E0B2D9010EEF6E1200AED97E
:100DE000EF6A12000901A26B01018A51220DF3CFB3
:100DF000A0F9F4CFA1F9000E0901A0270A0EA12342
:100E0000A8DAEECF98F9EECF99F9EECF9AF9EFCFB5
:100E10009BF9A6DAEECF9CF9EECF9DF9EECF9EF9C5
:100E2000EFCF9FF96DD9040E58D948DA01018F51DF
:100E3000090190270101905109019123000E92238D
:100E4000932308DBC4DADFDAE5DA01083AE17AEC69
:100E500015F001014B2B000E4C234D234E2380DA5D
:100E600012DA0901902B91239223932303DBF2DA08
:100E700077DA59DA69DA020B14E00A0EE66EE66AEE
:100E80008BC1E6FF8CC1E6FF2CD949D9125038D965
:100E900069D927D936DA0901120EA26F22D9020EBA
:100EA000DCD0040EA26F90C994F991C995F992C94A
:100EB00096F993C997F924D910D900DA12D99FDA93
:100EC000D9D042DA040B04E07AEC15F088EF09F08F
:100ED00017D9080E02D99451EE1801E0C9D09551E6
:100EE000EE1801E0C5D09651EE1801E0C1D097513F
:100EF000EE1801E0BDD001E0BBD08CDA02080AE1B7
:100F0000C2DA01E1B5D0B6DA62DA040EEF6EA0D92A
:100F10002CE3AED07FDA03082AE116DA020B01E1F6
:100F2000A7D0902B000E912392239323A3DAABDA60
:100F300006E0100EA26FD5D8040EEF6E13D0120E7D
:100F4000A26FCFD8020EEF6E942B000E952396233E
:100F5000972306DA94C9EEFF95C9EEFF96C9EEFF16
:100F600097C9EEFF75D901E383D061DA83D0C8D881
:100F7000040EB3D8EECF10F0EECF11F0B2D9E9D90C
:100F80001050EE1808E11150EE1805E11250EE185D
:100F900002E11350EE1802E07AEF15F06BDA3ADA5C
:100FA000040842E170DA09E09CD8C7D906E099D874
:100FB00049D997D814DA7FDAEF82C6D9010B15E048
:100FC0000901110EA26FCCD9EFCF94F9EE2AEFCF21
:100FD00095F9EE22EFCF96F9EE22EFCF97F9EF22B7
:100FE000B8D912D97ED80A0EEF6E32D941E279D83B
:100FF00059DA05E11CDA0901100EA26F3BD0090194
:10100000A26BAED99CC9EEFF9DC9EEFF9EC9EEFF53
:101010009FC9EEFF9ED998C9EEFF99C9EEFF9AC904
:10102000EEFF9BC9EEFF24D0F5D90A0805E17AEC62
:1010300015F029DA1FE01AD0EDD9050810E17AEC95
:1010400015F082D9010B16E00901100EA26F81D9AB
:10105000DBD819DA0BE145D8060EEF6E0BD0DAD9E2
:10106000060808E17AEC15F00EDA04E051D902D056
:101070007AEC15F00901A25100081EE2BAD8A2C903
:101080007EF190C97AF191C97BF192C97CF193C943
:101090007DF194C976F195C977F196C978F197C930
:1010A00079F12ED8DCD82CD8020E17D8DDD88BC118
:1010B00070F18CC171F1CFDC120001019151220D50
:1010C000F3CF10F0F4CF11F0000E10260A0E11220B
:1010D00010C0F3FF11C0F4FF1200E926000EEA224F
:1010E0001200A0C9E9FFA1C9EAFF120086C1E9FF09
:1010F00087C1EAFF12006DC9E9FF6EC9EAFF12005D
:101100008DC1E9FF8EC1EAFF12006DC9E9FF6EC90A
:10111000EAFF120083C9E9FF84C9EAFF1200EE5218
:10112000E9CF10F0EACF11F0E9CFE6FFEACFE6FF12
:10113000A3EC30F0126E060EE15E120088C1E9FFEA
:1011400089C1EAFF120000C9E9FF01C9EAFF1200E4
:10115000220DF3CFE9FFF4CFEAFF000EE9260A0ED5
:10116000EA221200EECF10F0EFCF11F012006CC99E
:10117000E9FF6DC9EAFF1200EECF7AF1EECF7BF105
:10118000EECF7CF1EFCF7DF1120090C9EEFF91C957
:10119000EEFF92C9EEFF93C9EEFF120001C9E9FF0D
:1011A00002C9EAFF120081C9E9FF82C9EAFF120001
:1011B000EE52E9CF70F1EACF71F12BEF05F001C9E2
:1011C000E9FF02C9EAFF120081C9E9FF82C9EAFF0B
:1011D0001200EECF76F1EECF77F1EECF78F1EFCFD0
:1011E00079F112001D0E64C3EBFF1E0E65C3EBFF09
:1011F00012000101806B816B01017F69120002C93D
:10120000E9FF03C9EAFF1200EF2AEECF90F9EF22BF
:10121000EECF91F9EF22EECF92F9EF22EFCF93F9D3
:10122000120002016C6F6D6B7FC16BF22AEF17F039
:1012300020C9E9FF21C9EAFF12000201696F6A6B48
:1012400017EF17F00F0EEB5002015A6F72EF15F007
:101250000101000ED8808F55000E90551200EECF80
:1012600074F1EDCF75F11200EECF72F1EDCF73F1A5
:101270001200220DF3CF00F9F4CF01F9000E002780
:101280000A0E012312004BC1EEFF4CC1EEFF4DC10F
:10129000EEFF4EC1EEFF1200100EEB6A110EEB6A6C
:1012A000280E02016C6F6D6B12007851F00BE84252
:1012B000E842E842E842040DF3501200EECF90F904
:1012C000EECF91F9EECF92F9EFCF93F91200EE6ADB
:1012D000EE6AEE6AEE6A1200CA0E105C030E115836
:1012E0001200EECF12F0EFCF13F0120082C1E9FF2F
:1012F00083C1EAFF12000F0EEB5002016B6F2AEF61
:1013000017F00D0E10C0EBFF0E0E11C0EBFF120018
:10131000A0C988F1A1C989F1CCEF06F0700EEE6E7C
:10132000170EED6E1200EE2AEE22EE22EE221200D1
:101330006CC1E9FF6DC1EAFF12000F0EEB50FF0810
:101340001200210E6DEF08F0DBDE0D0EC6DEEF5051
:101350001200C7DE180E6DEF08F0BFDE3DEF0AF099
:10136000C0DE37EF0AF0B9DEEECFDAF2EECFDBF215
:10137000EECFDCF2EFCFDDF279EC24F004C010F018
:1013800005C011F006C012F007C013F076EF08F0A8
:10139000A4DEB2EF08F0010EA0DE07C9EFFF76EF82
:1013A00008F09BDEE552E750EF6E76EF08F095DE31
:1013B000EFCF07F976EF08F090DE04C0EEFF11C022
:1013C000EEFF12C0EEFF13C0EEFF76EF08F089DEED
:1013D0001C0E83DEEF6A85DE05DF71EF08F00F0E6D
:1013E0007CDEEF681200180E78DEBCEF08F00D0E00
:1013F00074DE2FEF09F00B0E70DE34EF09F0EE52C1
:101400004ED867EF09F01F0E68DE8EEF09F07DDE23
:1014100037EF0AF066DEEF501200A9DE100E5DDE37
:1014200001015E51120067DE1C0EEB50120043D822
:10143000EF8657DE120E8FC1EBFF130E90C1EBFF4C
:101440003AD8EF8412007DDFEF501200100EA0DFBB
:101450006CEF09F085DFEECF94F9EECF95F9EECF82
:1014600096F9EFCF97F91200AADEA1EF09F0140E5A
:101470006DEF08F06EDFC5EF08F0010E2EDEEF50C5
:10148000E66E76EF08F060DF100B120087DEA1EF4A
:1014900009F023DECBEF09F0120E6DEF08F0060E17
:1014A0006DEF08F0D0DF080B120034DEA1EF09F079
:0C14B00045DEA1EF09F015DEA1EF09F008
:0414BC000B01AA6B0B
:1014C00064C3A4FB65C3A5FB0901036B080E035DA0
:1014D00015E2500E01014F6F506B6EEC00F0E66E9E
:1014E0000901E3DBA6EC0EF0E0DB020EC0DBEF6AE5
:1014F000DCDB090EBCDBEF6A032BE8D71200ABCBB9
:1015000000F9ACCB01F9090100C9E9FF01C9EAFF03
:10151000002B000E0123EF502E0807E000C9E9FF61
:1015200001C9EAFFEF50EFE10A0C026B0251106EA5
:10153000116A100E105C000E115814E20251A0DB6B
:1015400000C9E6FF01C9E6FFF1EC30F0136E050EAD
:10155000E15E1350000903E1090102511200090183
:10156000022BE4D70A0CBFDB04E0200E0901005D6A
:10157000FAE00901016B2B0E0901005D02E1200E6A
:10158000006F2F0E005D1FE05C0E005D1CE0200E62
:10159000005D1BE03F0E005D18E00D0E005D15E0E4
:1015A0000A0E005D12E00C0E015D0DE2610E005DA1
:1015B00005E300517A0802E3200E005F0151012B80
:1015C000AADB00C9EFFF8FDBD6E109010151A3DBE4
:1015D000EF6A090101510CE1D50E106E670E93DB25
:1015E000AECBE6FFAFCBE6FF07EC31F0050EE15ED8
:1015F0003F0E0901005D01E1010C000C0B01A4513B
:101600000301645D106E65510B01A555116EE00E6E
:10161000105C2E0E115801E3AA6B0901876B080EAE
:10162000875D06E287C9B0FB04D80901872BF7D78D
:1016300012000B01B0510A0DF3CF7CF9F4CF7DF904
:10164000540E09017C270B0E7D23010E7A6F0901D0
:101650007A5101E182D17A6B05DB64DB0AE17CDB44
:10166000EF50020B01E0AFDB77DBEF9479DBEF6A41
:101670001200F8DA020EEB50070AE9E0010A01E174
:101680005CD1030A01E12DD1010AE1E0070ADFE0A4
:10169000010A01E118D1030A01E1D6D0010AD7E11C
:1016A000E1DA4DDBD4E00901010E7A6F64C3A4FBDB
:1016B00065C3A5FB51DBEF6A6ADB0B01B66FAAD9E4
:1016C0000901796F49DBEF9462DB0101916F5DECF9
:1016D00008F067DBEE52060ECADA0B01A651EE18CF
:1016E00020E1A751EE181DE1A851EE181AE1A95109
:1016F000EE1817E116E1AA5102E02EDBEF84020E8C
:10170000AA5D02E0000E01D0010E106E25DB105024
:10171000010BF36EF346F346F346F70EEF14F310A6
:10172000EF6E0901795101E089D00B016C0EAE6FAB
:10173000090EAF6F2CDB0B01AD6F15DF0901806F58
:10174000580E6C5D15E108DBEF50040B11E10A0E39
:10175000E66EE66ADF0E106E670ED5DA6C0EE66E88
:10176000090EE66ECEEC30F0136E070EE15E1350FC
:101770000B016C0EAB6F090EAC6FC1DEE66EEADAE0
:10178000E5DA090180510BE001016C0EE96F090EE9
:10179000EA6F7CC9E7F17DC9E8F1A3EC10F018DB32
:1017A000DFDA050EEF6EE6DAD1DA00DB106E060E38
:1017B000105C30E312DB04082DE36C0EE66E090EBC
:1017C000E66E20EC31F0E552E552F3CF7BF905DB14
:1017D000030802E3030E01D0020E09017B5FFDDA6C
:1017E0000B0FE66EB7DAB2DAF8DA4ADA7B51146A2E
:1017F0006C0F136E090E142213C0E6FF14C0E6FF2F
:1018000007EC31F0156E050EE15E1550B3DAE552C6
:10181000E750EF6ECBDAFF0803E1D3DAEF6A06D0C8
:10182000C5DAFE0806E1CDDA030EEF6E99DA050E91
:1018300082D092DAEF8294DA010E7DD0790501E050
:1018400006D78EDA030E77D0B5DA01E100D70901A9
:10185000010E7A6F0B015E0EBB6F670EBC6F4EDA26
:101860000B016E0EBB6F670EBC6FA7DA73DAEF3435
:10187000EA6AFE0BEA36E96E6E0EE926020EEA22ED
:10188000EECFBBFBEDCFBCFB39DA64DAEFCF10F063
:101890000B0E105C06E30B017D0EBB6F670EBC6F79
:1018A0008CDAB0CBB9FBA6D998DA060803E154DA92
:1018B000EF8002D051DAEF90D5D9030ED8D9EF6A74
:1018C0004FDA020E38D0CED93ADA01E081DA7CC99B
:1018D000B7FB7DC9B8FBDCD8000901E1B8D673DAE3
:1018E00028D068DA01E1B3D66CDAEF34EA6AFE0B8D
:1018F000EA36E96E8E0EE926020EEA22EECF7EF976
:10190000EDCF7FF909017EC9F6FF7FC9F7FF7E2B76
:10191000000E7F230800F5CF7BF9F55005E07BC969
:101920005AF1A0D9D1D9EED732DA0101576F75EC4F
:1019300001F016DA060EEF6E8AD694D9F3D90AE0D2
:1019400039DA08E024DA0101566F35EC01F008DAE3
:10195000070EEF6E01DAEF947AD61200B4CBE9FFEE
:10196000B5CBEAFFEF0409011E6F1D6BEF6A1F6B19
:101970001E510B01EA6AB225E96EB351EA22EF6A01
:1019800009011F5141E101011C0E626F090E636FD5
:10199000B1CB61F1B9EC02F0000936E03D0E09016E
:1019A0001C5D0BE11C6B1E511D5D1EE21D29B4CB9D
:1019B000E9FFB5CBEAFFEF6E17D0260E1C5D02E102
:1019C000020E0AD0200E1C5D06E00D0E1C5D03E029
:1019D0000A0E1C5D04E1010E1F6F1C6B05D02B0E5F
:1019E0001C5D02E1200E1C6F1E511D5D06E2B2CB94
:1019F000E9FFB3CBEAFF1CC9EFFF0B01B22B000ECE
:101A0000B32309011D2BBCD709011F5101E1000CB3
:101A10001F0512000901056B040E055D19E2055151
:101A20000101626F636B000E6227090E6323B6CB60
:101A300061F1B9EC02F000090BE009010551052B39
:101A4000EA6A000FE96E090EEA22EF502008E4E18D
:101A500009010551EA6A000FE96E090EEA22EF6AF0
:101A6000470E005D07E1450E015D04E1540E025D85
:101A700001E1000C500E005D0AE14F0E015D07E12F
:101A8000530E025D04E1540E035D01E1010C020CF2
:101A9000F2D813D901E1A6D00901856BECD8030E69
:101AA000EB50040818E0E7D814D9400B0DE1E3D857
:101AB000010EEB500201386F8FEC23F00901866FA5
:101AC000DAD807D9200B07E0D6D8EF500101576FBD
:101AD00075EC01F0010CCFD8090EC9D8EF50010BFD
:101AE00001E17BD0C8D8030EEB50040A50E0070A8E
:101AF00034E0010A1BE0030A0BE0010A6BE1250E4A
:101B0000865D03E131D9010E26D0010E856F62D0CA
:101B1000250E865D03E1010E856F5AD029D9030E8B
:101B2000A6D886C9EFFF20D9020E15D0610E865DBA
:101B300002E3270E04D0410E865D02E3070E865FA6
:101B4000300E865D100DF350E66E12D9020E8FD85E
:101B5000FDD80AD9030EEF6E3DD0610E865D02E31B
:101B6000270E04D0410E865D02E3070E865F300E1D
:101B7000865D106EFDD8020E7AD81050EF12F4D8A0
:101B8000040EEF6E78D873D8EE6AED6A23D00101A7
:101B9000860EED6F090EEE6FB7CBEBF1B8CBECF123
:101BA00040EC11F0F3CF10F0F4CF11F0E1D8F3CF07
:101BB000EEFF11C0EDFF0901010E856FD9D8FF0EB0
:101BC000EE1808E1FF0EED1805E1865101E1856B85
:101BD000CBD8EF6A855101E15BD786C95AF14BD862
:101BE00073D856D748D8010EEB500201376F68EC16
:101BF00023F0000C0B01B9510A0DF3CF85F9F4CF96
:101C000086F9540E090185270B0E862301010D0E5E
:101C1000C1D801010A0ECAEF0EF00B01BA510A0D2C
:101C2000F3CF85F9F4CF86F9540E090185270B0E01
:101C30008623BBCBF6FFBCCBF7FF0800F55011E0C5
:101C40000B01BBCBF6FFBCCBF7FFBB2B000EBC23BD
:101C50000800F5CF5AF185C9E9FF86C9EAFF34D8F3
:101C6000E8D712007CC9E9FF7DC9EAFF1200E92626
:101C7000000EEA221200B7CBE9FFB8CBEAFF120050
:101C8000040DF3CFF6FFF4CFF7FF1E0EF626670E16
:101C9000F722F6CF10F0F7CF11F0126A10C0E6FF6E
:101CA00011C0E6FF12C0E6FF120003510A0D79D8F9
:101CB000540EE9260B0EEA221200EF500101586F74
:101CC000D9EC01F000091200EF500101596FF2EF59
:101CD00001F0010EEB50080D64D8000EE926020E4B
:101CE000EA22EF5012000101000E626F090E636FCD
:101CF000ADCB61F1B9EC02F0000912005ED8B0CBB7
:101D0000B9FBFAEF0DF0116E126A10C0E6FFE66E35
:101D100012C0E6FF12000B01EA6AAE25E96EAF5170
:101D2000EA221200EF500101556F2CEC01F000097E
:101D30001200010EEB500201366F60EF23F0EF50FE
:101D40000101696F44EC03F000091200E552E7500D
:101D5000EF6E120036D844D085DF090E37EF0EF053
:101D600081DF020E37EF0EF086DF030E37EF0EF045
:101D700082DF36D00201356B02016C0E336F090E23
:101D8000346FC3EC22F0E66E6DDFEE5212006ADFB4
:101D9000EF5012005A6F85C9E9FF86C9EAFF64EF68
:101DA0000EF0F3CFE9FFF4CFEAFF12005BDF010E84
:101DB000EB50120057DF5DEF0EF0B0CBBAFB0DEF2A
:101DC0000EF050DF0DD0C8DFEF924CDF99EF0EF030
:101DD000DEDF0101606F9BEF02F0BCDFEF5012000D
:061DE000040E37EF0EF0C7
:0A1DE600120053EC13F0040B06E0AA
:101DF00053EC13F0080B01E0020C010C000C09017C
:101E00001C6B1D6BE2C1E9FFE3C1EAFFEF506B08F9
:101E100001E080D00901010E206F0201210EE76F61
:101E2000090EE86F010E0101E2250201E56F000EC7
:101E30000101E3210201E66F7EEC25F0000903E1D8
:101E4000F36AF46A7FD1E4C1E6FFE5C1E6FF5EEC28
:101E50002BF0E552E552F3CF22F909012151110887
:101E600004E2160E0901215D05E109011C83090147
:101E7000206B43D009012151150809E3130E090114
:101E8000215D04E009011C8F0901206B36D0090196
:101E900021511A0801E331D0090121511E0801E343
:101EA0002CD009012151220817E31F0E0901215DE1
:101EB00004E0210E0901215D07E109012251080812
:101EC00002E30901206B02D00901206B09012051B6
:101ED00002E109011C8511D009012151300805E3F7
:101EE00009011C870901206B08D009012151320822
:101EF00004E309011C890901206B0901205109E152
:101F00000101E65106E022C9A8FF21C9D7F299ECE8
:101F100031F013D1E2C1E9FFE3C1EAFFEFCF10F0E6
:101F2000610E105C01E2B5D0E2C1E9FFE3C1EAFF56
:101F3000EF50670801E2ADD0E2C1E9FFE3C1EAFF7B
:101F4000EF50640807E0E2C1E9FFE3C1EAFFEF50A8
:101F5000650803E1F36AF46AF5D0E2C1E9FFE3C181
:101F6000EAFFEF509F0F09011E6F1F6B890E0901D9
:101F70001E270F0E09011F23010E0101EA6AE22547
:101F8000E96EE351EA22EF5014E10201200EE76FFF
:101F9000090EE86FE4C1E5F2E5C1E6F27EEC25F05A
:101FA000000906E01EC9E9FF1FC9EAFF20C9EFFFCB
:101FB0006FD0010E0101EA6AE225E96EE351EA22DF
:101FC000EF50780833E1020E0101EA6AE225E96E7A
:101FD000E351EA22EF50D00F106E010E105204E0D0
:101FE000E846FE0B1006FCE10901206FE4C1E9FFA1
:101FF000E5C1EAFFEF5031080AE10901201D106E2A
:102000001EC9E9FF1FC9EAFF1050EF160ED0E4C148
:10201000E9FFE5C1EAFFEF50300807E11EC9E9FF1B
:102020001FC9EAFF09012051EF1232D0010E010150
:10203000EA6AE225E96EE351EA22EF50D00F106E12
:10204000010E105204E0E846FE0B1006FCE1090107
:10205000206FE4C1E9FFE5C1EAFFEF5030080AE173
:102060000901201D106E1EC9E9FF1FC9EAFF1050AB
:10207000EF160ED0E4C1E9FFE5C1EAFFEF503108E9
:1020800007E11EC9E9FF1FC9EAFF09012051EF124C
:1020900054D0E2C1E9FFE3C1EAFFEF506C082DE143
:1020A0000101E65129E0010E0101EA6AE225E96E2B
:1020B000E351EA22EF50610A11E0030A01E01CD06B
:1020C0000201080EED6FE4C1EBF2E5C1ECF23E0E49
:1020D0000201E96FEA6BA3EC25F00ED00201080EB5
:1020E000ED6FE4C1EBF2E5C1ECF2350E0201E96FF0
:1020F000EA6BA3EC25F000D020D0E2C1E9FFE3C1F8
:10210000EAFFEF506D0819E10101E65116E0E4C164
:10211000E9FFE5C1EAFFEF50720A01E00ED0D3EC0F
:1021200016F0FF0E986E966E956E936E000E866E8C
:10213000846E836E816EFF0000D01CC9F3FF1DC941
:10214000F4FF00D012000901146B156B186BE7C186
:10215000E0F1E8C1E1F148DE0901196F140E166FD4
:102160000B01160EB46F090EB56F0B01000EB26FA6
:10217000090EB36FB1DAEF500B01B16FAEEC0CF09A
:102180000901176F182B1B6B6C0E005D36E10151B6
:10219000750A2BE0050A45E1010E1B6F3E0E54DA6D
:1021A00040E1020E0901185D3CE1010E1A1539E00B
:1021B00093DAEF500101916F5DEC08F0F3CFE9FF86
:1021C000F4CFEAFFEE52060E83DAEECFA6FBEECF97
:1021D000A7FBEECFA8FBEFCFA9FB0B01010EAA6F67
:1021E00043DAEF8441DAEF961CD0010E1B6F350EF7
:1021F0002BDA17E109011A8114D06D0E005D11E18F
:1022000019510FE01651EA6A000FE96E090EEA2231
:10221000EF506F0A06E1010E1B6F0B01AA6B24DA67
:10222000EF9409011B5115E119C9E6F1165101019D
:10223000E46FE56B000EE427090EE5230101000EB3
:10224000E26F090EE36FDBDDF35009011413F45064
:102250001513175101E082D71451020B01E012004F
:102260001451040B02E0ADEF31F01451080B02E001
:10227000FCEF31F01451100B02E028EC32F01200A8
:10228000F7D9020E25DAEFCF01F9F2D9030E20DAE1
:10229000EFCF02F9EDD9EECF07F9EDCF08F913DA58
:1022A000EF6AEBC1E0F1ECC1E1F19EDD0901096FDC
:1022B000610E025D6DE3025168086AE3006B610E16
:1022C000025D066F070E0115106E010E105204E03C
:1022D000E846FE0B1006FCE10901056F0651036F8D
:1022E000046B920E03270F0E0423D0D909E1065187
:1022F000036F046B890E03270F0E0423008107D0A0
:102300000651036F046B800E03270F0E0423F00E9B
:102310000115066FE85004E1B9D934E0310E35D02B
:10232000100E065D0CE1B2D905E10101BE0EF26F9F
:10233000680E02D10101BB0EF26F680EFDD0200EB7
:10234000065D03E1010E001506E0300E065D08E1B2
:10235000010E001505E0080E011501E1D8D0E8D006
:10236000400E065D08E1010E001505E00101A10E19
:10237000F26F680EE1D0500E065D01E0E6D0010E6E
:10238000001502E0300E01D0310E9DD9EF6EDDD088
:102390006B0E025D0AE1095101E1D7D001C9D6F205
:1023A0008FEC31F00101FC6F62D06C0E025D42E1F6
:1023B00009512CE00151040A24E0060A1DE0030A39
:1023C00016E0010A01E0C1D009050CE1350E01015A
:1023D000F76FF86BEDC1F5F1EEC1F6F107C9F4F155
:1023E000C7EF12F00101250EF26F500EA5D00101CA
:1023F000C60EF26F690EA0D00101CC0EF26F690E0D
:102400009BD00101220EF26F500E96D00151030AAB
:1024100008E0030A01E099D001011C0EF26F500E92
:102420008BD0095102E1300E01D0310E066FE8CF9A
:10243000FCF11DD06E0E025D01E087D0006B0F0E27
:102440000115106EC11C0F0B105C01E20083F00E31
:102450000115066FE85005E10101880EF26F680E64
:102460006BD0100E065D0BE126D9EFCFFCF1EDC16C
:10247000FAF1EEC1FBF107C9F9F1E8EF12F0200E15
:10248000065D39E118D9EFCF06F90751081120E1AF
:10249000330E03D90750300F0101DA6F2E0EDB6FB8
:1024A000330EFBD803C006F9090103500A0DB8D852
:1024B0000101DC6F0A0EF1D807C006F909010750C7
:1024C000640DAED80101DD6FDE6B0901076B086B8F
:1024D0000751D5D8F8D8EF6E0751D1D836E007C9E3
:1024E00010F008C911F0072B000E082307C9F3FFED
:1024F00008C9F4FF1200300E065D03E1020E00155C
:1025000006E1500E065D08E1020E001505E101012D
:10251000B20EF26F680E10D0400E065D03E1020E9F
:10252000001506E1600E065D10E1020E00150DE1DA
:102530000101B70EF26F680EF36FEDC1F0F1EEC15D
:10254000F1F107C9EFF1A8EF12F0F368F468120097
:102550000101EF51F76AF225F66EF351F7220800F8
:10256000F550F0C1E9FFF1C1EAFFEF6EF0C1E9FFFC
:10257000F1C1EAFFEF5003E1F368F4681200EF2BBA
:10258000EF51116AEFC1F3FF11C0F4FF1200010116
:10259000F451F72509010A6F000E0101F821AA6E16
:1025A0000AC9A9FF3F0EA616A680A850F5C1E9FFEB
:1025B000F6C1EAFFEF6EA85003E1F368F468120079
:1025C000F42BF451116AF4C1F3FF11C0F4FF1200AF
:1025D0000101F95110E1DA0EE66E010EE66EFC51D2
:1025E000E66EE66AD3EC2BF0E552E552E552E55291
:1025F0000101DF6BF96BF95142D8FAC1E9FFFBC168
:10260000EAFFEF6EF9513BD803E1F368F46812007A
:10261000F92BF951116AF9C1F3FF11C0F4FF12004F
:10262000F3CF10F0F4CF11F0330E0B6E0C6AF3CF32
:1026300006F0F4CF07F097EC34F006C010F007C0B6
:1026400011F0300E062412000201F06FF16B090147
:1026500016510201EE6FEF6B000EEE27090EEF230D
:10266000DBEC25F00009120037D8090E68EF13F0F3
:10267000EBC1E9FFECC1EAFF040E68EF13F0EA6A70
:10268000DA0FE96E010EEA22EF50120003C9E9FFEA
:1026900004C9EAFFEF5005151200106E0C6E06C952
:1026A00007F0BEEF34F0E0C1E9FFE1C1EAFF090E37
:1026B0000FD8EF5012000F0E0115EA6ACA0FE96E2B
:1026C000020EEA221200EDC1E9FFEEC1EAFF12009C
:1026D000E926000EEA221200E7C1E9FFE8C1EAFF9D
:0226E0001200E6
:0E26E200966A8688988802014A6B4B6B4C6B97
:1026F0004D6B4E6B4F6B0901006B0051106E116AF0
:10270000D890115004E6010E105C000E115814E22E
:102710000051040DF3CF10F0F4CF11F0400E10264D
:10272000000E11220051AFDB10C0EFFF0051ABDBF8
:10273000EE52EF80002BE1D71B6A0201496933DBBF
:10274000B7DB02011F0EB1DB0201656F02011F0E34
:10275000A9DBAEDB0201210EA0DBAADB0201080E21
:10276000656F02010E0EC7DB0A0EC5DB0B0ED1DB57
:10277000040E656F02010C0ECCDB020E656F0201C8
:102780000D0E90DBDBDB8EDBB1DB010EC2DB600EFE
:10279000656F0201020E86DBA9DB030EBADB6569F9
:1027A0000201070EA8DB0F0EB4DB610E76DBBCC2A4
:1027B00065F20201010E76DBBDC265F20201020E76
:1027C00071DBBEC265F20201030E6CDBBFC265F2B3
:1027D0000201040E67DBC0C265F20201050E62DB76
:1027E000C1C265F20201060E5DDB0901006B080E35
:1027F000005D0AE202016569080E09010025020177
:1028000051DB0901002BF3D771DB070E4BDB440EC4
:10281000186E0201220E41DB51DB0D0E7ADBE00E59
:102820003CDB0201C00E656F0201010E64DB040E89
:1028300062DB010E6EDB200E4DEF17F002010D0E74
:1028400070DB02014A2711504B2302010E0E69DB97
:1028500002014C2711504D2302010F0E62DB0201D1
:102860004E2711504F231200020149511B5C09E110
:102870000201666BB3DA040B03E10201496964D318
:10288000000C62D325DB86A8FED78D8C6B0E8D6E77
:10289000836A8D9C86A8FED722DB86A8FED78D8C06
:1028A000670E8D6E400E836E8D9C86A8FED78D8C34
:1028B000700E8D6E50C283FF8D9C86A8FED78D8CC6
:1028C000192A000E1A22120002015351541101E17B
:1028D0001200010E5315106E116A53511024090194
:1028E0003E6F02015451112009013F6F956A670E36
:1028F0008D6E400E836E8D9C86A8FED78D8C6A0EE1
:102900008D6E3EC983FF8D9C86A8FED78D8C6B0E85
:102910008D6E3FC983FF8D9C86A8FED7E0DA86A81E
:10292000FED78D8C02015351192654511A22700E74
:102930008D6EE4DA86A8FED78D8C53C23CF954C262
:102940003DF90901010E3C5F000E3D5B09013CC9E8
:1029500010F03DC911F03C07000E3D5B1050111006
:1029600030E0080E3C5D000E3D5926E389DA86A86A
:10297000FED78D8C85DA86A8FED78D8C81DA86A865
:10298000FED78D8C7DDA86A8FED78D8C79DA86A865
:10299000FED78D8C75DA86A8FED78D8C71DA86A865
:1029A000FED78D8C6DDA86A8FED78D8C080E0901B6
:1029B0003C5F000E3D5BD5D763DA86A8FED78D8CD1
:1029C000C5D7120085DA86A8FED78D8C6B0E8D6E6A
:1029D000836A8D9C86A8FED78D8CFF0E195C1DE145
:1029E0005F0E1A5C1AE109013269336932C967F274
:1029F00033C968F201DA66DA86A8FED78D8C020147
:102A0000100E53DA0901316F326B440E336F32C945
:102A100067F2E8CF68F2F0D910D054DA86A8FED772
:102A20008D8C9568700E8D6E8D9A86A8FED783CF9B
:102A300031F98D8A192A000E1A220901315112002A
:102A400057C2B5F958C2B6F902015751581103E1FE
:102A5000F36AF46A1200956A6A0E8D6EB5C983FF37
:102A60008D9C86A8FED78D8C6B0E8D6EB6C983FFAC
:102A70008D9C86A8FED78D8C25DA86A8FED78D8CF6
:102A80000901B5511926B6511A22600E1A5C02E3EB
:102A90001C0E1A5E9568700E8D6E0901B5C910F096
:102AA000B6C911F0B507000EB65B105011100FE05B
:102AB0008D9A86A8FED7020155C2E9FF56C2EAFFE9
:102AC000552B000E562383CFEFFF8D8AE6D757C2D2
:102AD000F3FF58C2F4FF120002015951D4D9EE524B
:102AE000EF90120002015A51CED9EE52EF805AC235
:102AF0001BF0120018C036F90901010E356FE8CF3E
:102B000067F218C068F278D95DDF0901346FE8CF49
:102B100065F20201030E52EF17F0FED90901006FB2
:102B20000201200EBAD918500901005D05E2600EBD
:102B3000D8801854002502D01850005D016FE8506D
:102B4000106E116A1C0ED8801056000E115610C05F
:102B500001F910C003F9026B02C9F3FF10C0F4FFC2
:102B600012000201E00EE5D90901006F0201200EFA
:102B700094D909010051040B01E0000C010C5DC265
:102B8000E9FF5EC2EAFFEF68C7D90901126F0201CF
:102B9000200ECFD90901136FDCD9100B37E00201E9
:102BA000666B1CD9040B0901176F0201210E75D940
:102BB000020EE66E80EC34F0E55280D90A0E9BD905
:102BC0000B0E70D90901175108E0C3D90A0B02E0B6
:102BD000000E01D0010E0901176F0201020E656F90
:102BE00002010D0E96D9220E58D912C918F082DFB3
:102BF000020165690201070E7ED90D0E53D9090144
:102C0000175103E00201260E48D9000C09011351A7
:102C1000125D67E013C915F9146B14C967F213C983
:102C200068F2EAD8120E0201576F586B0201000ECB
:102C3000556F090E566F04DF09010051010B4EE07C
:102C4000400E025D000E035949E3EE0ED880025596
:102C5000050E035543E3600E015D40E20151106E25
:102C6000116AD890115004E6440E105C000E115801
:102C700035E310C9D8F211C9D9F274EC24F0F3CFBE
:102C800010F9F4CF11F9060EE66EE66A0A0EE66E4A
:102C9000090EE66E5BC2E9FF5CC2EAFF5BC210F0A0
:102CA0005CC211F05BC2E6FF5CC2E6FFA3EC30F051
:102CB000126E060EE15E1250080E0901115D0BE165
:102CC000105103E0060E105D06E15DC2E9FF5EC231
:102CD000EAFF10C9EFFF13C918F0010C12C918F070
:102CE00009DF000C02010A0E656F0201070EDAD837
:102CF0001DD9EFCF41F90901406B40C967F241C9C5
:102D000068F27AD8060E0201536F546B5FC251F21B
:102D100060C252F2D9DDBCC250F2B4DDBDC250F285
:102D2000B1DDBEC250F2AEDDBFC250F2ABDDC0C2FB
:102D300050F2A8DDC1C250F2A5DD0201615103E1EC
:102D40000901426B03D00901060E426F0201080E11
:102D5000506F98DD42C950F295DD0E0E02016227D8
:102D6000000E63233C0E625D000E635903E23C0ECD
:102D7000626F636B62C240F963C241F962C265F27D
:102D80000201050E8FD841C965F20201060E52EF0D
:102D900017F0D4D8BED8240E80D81BC049F2C6D8AC
:102DA000EE52EF8012009568600E8D6E8D8C8D8ACC
:102DB0008D8E966A0A0EE66ED8EC34F0E55278D81D
:102DC0008D9E1200600E020164118D6E65C283FF3C
:102DD000956A8D9C86A8FED78D8C12009568600E32
:102DE000020166118D6E8D9A86A8FED783CF37F9C2
:102DF0008D8A09013751120067C219F068C21AF0B2
:102E000067C265F20201080E4DD868C265F2020180
:102E1000090E52EF17F00201090E47D80901016FA0
:102E20000201080E42D8F36E01C9F4FF120018C067
:102E300023F90901120E226F0201695109012227AB
:102E400002016A510901232322C967F223C968F2EA
:102E5000FCEF16F06BC21BF069D8EFCF0DF909013A
:102E60000E0E0C6F02016C5109010C2702016D510D
:102E700009010D230CC967F20DC968F2FCEF16F0C9
:102E800002017EEF17F0E96EEA6AD890E936EA3679
:102E9000460EE926020EEA221200656F0201646BFB
:102EA000E2EF16F0646FE2EF16F0666FEEEF16F0E9
:102EB000050EE66E80EC34F0E55212000201656BFF
:102EC00002011200600E8D6E0A0E836E8D9C120040
:102ED000956A6A0E8D6E010E836E8D9C12008D8C2C
:102EE000600E8D6E120E836E8D9C12000201440ED8
:102EF000656F02011200D6DF5EEF17F051C2E9FFE5
:102F000052C2EAFF512B000E5223EF50836E8D9C6C
:102F10001200C8DF020112000201600EBEDFA9EF3D
:102F200017F0C3DF106E116AE85012001B5043EF18
:102F300017F0B3DF0201030E55EF17F0F7DFEFCF05
:102F400065F20201040E1200F1DFEE52EF50010BA8
:0A2F500012000201070E55EF17F002
:062F5A000901006B020EEC
:102F6000005D07E200513BDB00512DDBEF90002BB1
:102F7000F6D712000901000E016F010E026F006BFF
:102F8000020E005D43E2DCDA0C0EC7DACADA126A1E
:102F9000136A105011101210131032E1D1DA0C0E16
:102FA00029C1EBFF0D0E2AC1EBFF01012B512C11A2
:102FB00011E00A0EE66EE66A2BC1E6FF2CC1E6FFC1
:102FC000BFDA01C910F002C911F001C9E6FF02C958
:102FD000E6FFD8DAB5DA0A0E2DC1EBFF0B0E2EC1D3
:102FE000EBFFAEDA0E0EEB6A0F0EEB6AA9DA100EEB
:102FF000EB6A110EEB6A00C928F1090100511200B9
:10300000140E0127000E0223002BBAD7FF0C01017A
:103010002F51EFEF1AF0020E0101305D04E230C1D2
:1030200028F134EF14F0000C01012851140DF3CFF6
:103030000AF9F4CF0BF9000E09010A27010E0B2340
:10304000CADAEE50ED1004E190DA94DA8EDA87DA1B
:1030500031C150F242EC14F0BEDAEE2AEF22BBDAB4
:10306000C4DA01E346D8010C01012851140DF3CF55
:103070000AF9F4CF0BF9000E09010A27010E0B2300
:10308000A6DAEE50ED1004E151DA74DA4FDA67DABD
:103090009EDA01013451EE24106E3551EE20116E8E
:1030A000D60ED8801054030E11540AE290DAEECFF7
:1030B00034F1EFCF35F1D60ED8803457030E3557A3
:1030C00034C153F235C154F232C151F233C152F21C
:1030D00064EC14F07CDA01013451EE263551ED2216
:1030E00076DA83DA01E305D834C1F3FF35C1F4FFA2
:1030F000120001012851140DF3CF08F9F4CF09F99A
:10310000000E09010827010E092315DA0C0E05DA55
:1031100040DAF3CF00F9F4CF01F90DDA0A0EFDD948
:1031200038DAF3CF02F9F4CF03F905DA0E0EF5D948
:10313000EECF04F9EFCF05F9080E09010427000EC0
:103140000523066B076B140E02016C6F6D6BF3D9D0
:1031500006DA04C957F305C958F30301110E566F77
:10316000EAD908C954F309C955F3DFEC26F004C9BC
:10317000D8F205C9D9F274EC24F0F3CF04F9F4CFF6
:1031800005F9080E0201536F546B0201000E516FD6
:10319000090E526F64EC14F0C9EC16F0CCD9120E83
:1031A000BCD9EF68C8D90E0EEB6A0F0EEB6A12009D
:1031B000020E0101365D0AE236C128F1FFD9D8803E
:1031C000EE54000EED5401E3000C010C000C17DA74
:1031D00001E1000C2851F7D9EF50010B01E013DA9F
:1031E000E2EC14F037C1E9FF38C1EAFFEF6E11DA03
:1031F000EE06EF5AE3D9EE50ED1002E17AEC15F04D
:10320000010CFDD903E1F36AF46A12002851DBD9FD
:10321000EF50010B01E0F7D9FCD983D93B51105C89
:103220003C51115805E2CAD9EECF3BF1EDCF3CF14C
:103230003BC157F23CC158F239C155F23AC156F27E
:1032400020EC15F0F3CF00F9F4CF01F9E2D9090130
:103250000051EE5E0151ED5AD2D902E17AEC15F03F
:103260003BC1F3FF3CC1F4FF1200C9D902E07AEC84
:1032700015F0CFD9EE6AED6A1200080E0201576F01
:10328000586B0201460E556F090E566F20EC15F073
:1032900046C95DF947C946F95DC947F948C95DF9AD
:1032A00049C948F95DC949F9080E106E09014B5129
:1032B000D880105403E24A055D6F02D04AC95DF917
:1032C000080E4B5D4A6F5DC94BF94CC95DF94DC99C
:1032D0004CF95DC94DF93DC1E9FF3EC1EAFF060E5B
:1032E0001CD9EECF4FF9EECF50F9EECF51F9EFCF19
:1032F00052F955D9EFCF53F9010E0FD9EFCF54F949
:103300004ED9020E0AD9EFCF55F949D9030E05D986
:10331000EFCF56F9576B110E586F41C159F942C1A1
:103320005AF941C1D8F242C1D9F274EC24F0F3CF7A
:1033300059F9F4CF5AF90C0E0201E06FE16B02016A
:103340004F0EDE6F090EDF6FA8EC24F0F3CF5BF9B0
:10335000F4CF5CF909015B1F5C1F1A0EFBD85BC937
:1033600050F242EC14F05CC950F242EC14F0140E2E
:10337000F1D841C1E2F242C1E3F204EC25F0F3CF0F
:103380005BF9F4CF5CF909014C51F31816E14D518A
:103390005C1913E13FC147F140C148F13DC145F11E
:1033A0003EC146F10101460E436F090E446F1CD821
:1033B00009014E6FFF0E4E5D03E17AEC15F0010C32
:1033C0004E51A1D8100EA9D84AC9EEFF4BC9EDFF46
:1033D0004E51F9D8EF80010C0101285194D8E9CF62
:1033E000F3FFEACFF4FF120009010169000E026F3A
:1033F000010E036F006B020E005D5BE2A6D80C0E9F
:10340000FAD8020E8AD8D5D80001125010184AE115
:103410001350111847E199D80A0EEDD8CAD81250A6
:1034200010183EE1135011183BE18FD8100E75D8DB
:10343000EECF14F0EFCF15F0166A176A145015107E
:10344000161017102DE145C1E9FF46C1EAFF060E2F
:1034500064D8EECF10F0EECF11F0ABD876D8060ED0
:103460005CD8EE50101808E1EE50111805E1EE504E
:10347000121802E1EE50131810E047C1E9FF48C1ED
:10348000EAFFE868EE180CE1E868EE1809E1E86880
:10349000EE1806E1E868EE1803E109010051120098
:1034A00000C901F90901140E0227000E0323002BA5
:1034B000A2D7FF0E015D24E00151140DF3CF02F9F4
:1034C000F4CF03F9000E0227010E03230A0EE66E65
:1034D000E66A45C1E6FF46C1E6FF37D802C910F0EB
:1034E00003C911F002C9E6FF03C9E6FF4BD85CD857
:1034F00018D82BD80A0E10C0EBFF0B0E11C0EBFF33
:10350000090101511200140DF3CFE9FFF4CFEAFFD6
:10351000000EE926010EEA221200E926000EEA2238
:103520001200EECF10F0EFCF11F012000AC9E9FF40
:103530000BC9EAFF120008C9E9FF09C9EAFF120036
:1035400001C9E9FF02C9EAFF120002C9E9FF03C984
:10355000EAFF12000201696F6A6B17EF17F0120E93
:10356000EB5002016B6F2AEF17F00AC9E9FF0BC994
:10357000EAFF1200120E1BC0EBFF1C0E02016C6F63
:103580006D6B1200A3EC30F0126E060EE15E12506D
:103590001200EECFD8F2EDCFD9F274EF24F03FC194
:1035A000E9FF40C1EAFF120043C1E9FF44C1EAFF5D
:1035B0001200EECF12F0EFCF13F012002851A3DF6C
:1035C000100E8DEF1AF09FDF130E8DEF1AF0AEDFA5
:1035D0000E0E8DEF1AF0C9DF0E0E8DEF1AF093DF8D
:1035E0000C0E9BDFEE6AED6A12009BDFD60E105CBC
:1035F000030E1158120091DF94DFD4EF1AF009D8AE
:10360000EE50ED1012002851DEDFEF901C0EAAEFF5
:083610001AF00101DEEF1AF0CF
:08361800070E0301755D01E1DD
:103620001200FF0E765D01E0A7DA03017669756B83
:10363000786B120003017551060A01E1A2D0030A5A
:1036400066E0010A59E0070A46E0010A33E0030A8E
:1036500027E0010A01E0120009010E690F691069F3
:1036600011691269136914691569166917690301EB
:10367000086B096B0A6B0B6B430E01012D6F2E6BF0
:1036800001010E0E2B6F090E2C6F440E0101296FE4
:103690002A6BBAEC17F00301766F62DA010E756FD0
:1036A00050DA140E105C000E115801E27DD00301B7
:1036B000020E3BD00301085109110A110B1133E12D
:1036C00076C330F10BEC18F000096EE00301010E37
:1036D0005FDA030E2AD061DA03E30301020E756F8D
:1036E00076C336F1D8EC18F000095EE063D8020822
:1036F0005BE10301040E756F76C330F10BEC18F03B
:10370000000952E00301030E43DA050E0ED076C322
:1037100036F1D8EC18F000092EE04CD80901186FEA
:10372000060E185D04E10301040E756F1200050E0C
:10373000185D26E121DA0301766912DA060E756F4B
:1037400008C3B8F209C3B9F20AC3BAF20BC3BBF299
:1037500010C3C2F211C3C3F212C3C4F213C3C5F241
:103760000CC3C6F20DC3C7F20EC3C8F20FC3C9F231
:103770007781782B120011DA17E30301020E756FBF
:103780001200DFD9640E105C000E11580DE304071F
:10379000000E055B065B075B04510511061107115E
:1037A00002E10301756BDCD912000301080E756F8D
:1037B000BCEF1DF00901026B03013C0E046F056BA9
:1037C000066B076BB0D9020E0901005D01E0EBD07A
:1037D000016B0F0E015D02E2EFD9FBD70101080E6C
:1037E000376F030EABD9090E376F030EA7D90A0E38
:1037F000376F030EA3D90B0E376F030EC6D909011D
:10380000016B080E015D02E2D7D9FBD7BCC208F9F3
:10381000BDC209F9BEC20AF9BFC20BF9C0C20CF998
:10382000C1C20DF9016B060E015D0EE27CD90901E2
:103830000151EA6A080FE96E090EEA22EF50005DB5
:1038400001E0D3D0012BEFD7016B0151106E116A4B
:10385000D890115004E6CE0E105C000E115802E212
:10386000ABD9F3D7036B5FD909010051330A62E08A
:10387000CC0A5DE0C90A47E0350A23E0020A0DE000
:10388000340A01E07DD04FD90901000501E0ADD037
:103890000101020E376F090E48D072D901E0A5D0A0
:1038A0000101100E376F030E49D9110E376F030E49
:1038B00045D9120E376F030E41D9130E376F030E21
:1038C00034D05ED901E291D001010C0E376F030EA6
:1038D00035D90D0E376F030E31D90E0E376F030E2B
:1038E0002DD90F0E376F030E50D9040E0901005F5A
:1038F000090100510007000952E00101010E376F74
:10390000090E43D9F5D73CD970E10101070E376F95
:10391000090E14D9060E376F090E10D9050E376F30
:10392000090E0CD9040E376F090E2FD938D0010EAD
:10393000036F35D025D959E10101070E376F030E0A
:10394000FDD8060E376F030EF9D8050E376F030E3C
:10395000F5D8040E376F030E18D9D880080E03016E
:103960000455070E0555000E0655000E075517E2C3
:10397000080E045F070E055B000E065B075B0FD0A9
:103980000101000E376F090E00D90901005100072F
:10399000000905E00101010E376F090EF5D7090195
:1039A000035101E160D7020E025D09E104C900F391
:1039B00005C901F306C902F307C903F311D0000ECC
:1039C000E96E030EEA6EEE50041908E1EE50051997
:1039D00005E1EE50061902E1EE50071901E0026B15
:1039E00035EC19F009010251120035EC19F0000C08
:1039F0000101010E9ED8010E9CD8060E9AD8ABD8B4
:103A0000120E97D8230E95D8340E93D8560ECBD8D5
:103A1000800EC9D8A0D89FD8316B14EC18F00901DA
:103A2000196B0C0E195D02E2A0D8FBD7BCC231F1B4
:103A300014EC18F0BDC231F114EC18F0BEC231F133
:103A400014EC18F0BFC231F114EC18F0C0C231F11F
:103A500014EC18F0C1C231F114EC18F00901196B23
:103A60001951106E116AD890115004E6CA0E105CFC
:103A7000000E115802E279D8F3D70101630E59D82C
:103A8000820E57D8530E55D8630E53D8350E51D8E1
:103A9000010E316F14EC18F016C331F114EC18F06C
:103AA0000301160518E0085109110A110B1113E062
:103AB0000101360E7CD803C331F114EC18F002C3B7
:103AC00031F114EC18F001C331F114EC18F000C31B
:103AD00031F114EC18F00101370E2BD8020E29D861
:103AE000010E27D8030E316F14EC18F0030E0301FA
:103AF000165D13E10101320E5AD808C331F114ECFE
:103B000018F009C331F114EC18F00AC331F114ECC8
:103B100018F00BC331F114EC18F00101316914EC09
:103B200018F079EF18F00101000E376F090EC5EF9C
:103B30001DF0316F14EC18F00101120026D80101BC
:103B40001200030114510301645D106E65510301FD
:103B50001555116E1200316B14EC18F001011200B2
:103B600064C314F365C315F312000101316B14EC47
:103B700018F00901192B120076C32FF107EF18F086
:103B8000D2DF040E0901005D1200386FE7EF18F074
:103B9000166F2EDFE5DF03011200D3DF900E105CFD
:103BA000FF0E11581200C5DFD6DFABEF1DF0C1DFED
:103BB000040E316F14EF18F0B6DF0901012B12006B
:103BC0000001F35101E112000001FB0EF16F5C0EE8
:103BD000F26FE5EC32F000010B0EF16F5B0EF26F4D
:103BE000E5EC32F0F3C0B4F90901B451000814E275
:103BF000B451070B05E100012E0EED6F86EC32F09B
:103C000027DA02E057D908D0320EE66E80EC34F0A5
:103C1000E5520901B407E8D72DEF20F03CDAE7D9E7
:103C2000010EE926000EEA22E2D9020EE926000E74
:103C3000EA22DDD9030EE926000EEA223EEF20F04B
:103C40000901016B05DAFEE076EC32F00901006F44
:103C50000D0E005D17E00A0E005D14E0012B00015F
:103C6000F6C0E9FFF7C0EAFFF62B000EF72300C904
:103C7000EFFFF6C0E9FFF7C0EAFFEF6AF851F80777
:103C80000009E0E1090101511200F9C001F9FAC08F
:103C900002F90901036BF9C0E9FFFAC0EAFFEFCFAF
:103CA00000F9EF5021E02E0E0901005D11E1000145
:103CB000F9C0E9FFFAC0EAFFF92B000EFA23EF6A18
:103CC000AFD9032BD1D9F9C001F9FAC002F907D055
:103CD000300E005D03E30051390801E2000C0001E1
:103CE000F92B000EFA23D7D79BD9BED9030E0901B1
:103CF000035D01E0000C010CABD9FEE076EC32F084
:103D00000901006F310E005D05E3390E005D02E22E
:103D100000511200390CA1D9300E0001FD5DFF0FDA
:103D2000E96EEA6AD890E936EA362D0EE926030EE6
:103D3000EA22EECFF1F0EDCFF2F0E5EC32F0000147
:103D4000FD51380A01E1B5D00F0A01E1B0D0010AF6
:103D500001E1A1D0030A01E197D0010A54E0070A6A
:103D60004BE0010A42E0030A01E012000201330EB7
:103D7000D66F8FEC31F00901A16F0201340ED66FBE
:103D80008FEC31F00901A26F870EE66E090EE66E28
:103D9000A1C9E6FFA2C9E6FF87D9870EEF6F090E1A
:103DA000F06FD4EC32F029D9000947E0870EE66EB7
:103DB000090EE66E5EEC2BF0E552E552F3CFA1F969
:103DC000F4CFA2F9F3CFA8FF0201330ED76F99EC1D
:103DD00031F0A2C9A8FF0201340ED76F99EC31F07F
:103DE000A2C9C0F2A1C9C1F212000901B80E9F6FA9
:103DF000020EA06FA36B0ED00901C60E9F6F020EBC
:103E0000A06F0E0E06D00901C20E9F6F020EA06FAA
:103E10000A0EA36F9FC9F4F0A0C9F5F0FFDEEDD83C
:103E200000019B0EFB6F090EFC6F0001870EF96FFE
:103E3000090EFA6F2ADF00090BE10001B10EF16FE4
:103E40005C0EF26FE5EC32F003D9FEE076EF32F073
:103E50009FC9E9FFA0C9EAFF9BC9EEFF9CC9EEFF1D
:103E60009DC9EEFF9EC9EEFF9BC9A8FFEAD89CC979
:103E7000A8FFE7D89DC9A8FFE4D89EC9A8FF0901FB
:103E8000A351A32B020110D00201160ED66F8FECA6
:103E900031F0010906D00201160ED66F8FEC31F019
:103EA000FE0BA86E0201160ED76F99EF31F06FEF7F
:103EB0001FF012000001440EF16F5B0EF26FE5EC93
:103EC00032F01ADF0901B56F390EB55D03E0B5C9EF
:103ED000FDF021DF380E0901B55DECE112000901AA
:103EE000006B026BF8EC23F064C385F965C386F9B7
:103EF000090185510301645D106E65510901865504
:103F0000116E320E105C000E115809E364C385F97E
:103F100065C386F90001150EED6F86EC32F098D876
:103F2000E7E00901025162E193D8FBE076EC32F060
:103F30000901016F0051030A20E0010A1BE0030A96
:103F400014E0010502E1010E16D0040E015D09E145
:103F500041EC24F00001060E9BD80901010E026F0E
:103F6000E0D70001150E94D8DCD7060E046F036B62
:103F7000020E01D0030E006FD4D70351032BEA6A5F
:103F8000050FE96E090EEA2201C9EFFF0351106E19
:103F9000116A1134C6E210508008000E1154C1E2BB
:103FA000060E046F016B0151106E116AD89011500A
:103FB00004E6800E105C000E11580DE20151EA6A11
:103FC000050FE96E090EEA22EFCF45F210EC24F05E
:103FD0000901012BE8D70201376B68EC23F004C913
:103FE000EDF086EC32F00901006B9BD7010C46D84E
:103FF00000012E0E4DD84BEF20F00001290E48D8BD
:1040000000013A0E45D80001200E42D80001140EDE
:10401000F86F0001870EF66F090EF76F20EF1EF0A4
:1040200001C9E6FF02C9E6FF5EEC2BF0E552E5525E
:10403000F350E66EFBC010F0FCC011F00901035113
:1040400012000901A351A32B0201D76F99EF31F0A0
:104050000001EA510001EB5D120000010D0E18D8BD
:1040600000010A0E48EF20F00F011024E96E000E47
:104070001120EA6EE552E750EF6E1200EF50E66E47
:10408000E66A12D8000EEF6F090EF06FD4EF32F02F
:10409000ED6F86EF32F0000EE66E090EE66EF4C0AC
:1040A000E9FFF5C0EAFF1200D3EC2BF0E552E55230
:0840B000E552E5520001120087
:0840B800150E01014F6F506B62
:1040C0006EEC00F00101936F976BC56B926B140E51
:1040D000956F966B120093C155F12CEC01F000091D
:1040E00007E10101C56B070E996F976B926BA6D024
:1040F00093C169F144EC03F0000934E020DA0101D6
:10410000700E626F090E636F93C161F1B9EC02F03A
:1041100000090EE01F0E0101C55DF1E2C551C52B7E
:10412000EA6AA40FE96E010EEA2270C9EFFFE7D731
:1041300093C160F19BEC02F00A0E0901705D26E16B
:104140000101C551EA6AA40FE96E010EEA22EF6A85
:10415000C56B9BD9C6C1D8F1C7C1D9F15DD90101E1
:10416000996F14D00101975111E0D5510301645D9D
:10417000106E65510101D655116E500E105C460E41
:10418000115804E3DCD9020E996F976F0101975122
:10419000020A3EE0070A0DE0040A06E0010A54E1C3
:1041A0009A6BCDD9010E976FBED94EE00101050E75
:1041B000976FB9D92DE09AC1E9FFEA6AE9BEEA68CA
:1041C000D890E936EA36A20EE926020EEA22EECFB0
:1041D00071F9EDCF72F9090171C9F6FF72C9F7FFE4
:1041E000712B000E72230800F5CF70F9F55007E02F
:1041F00070C95AF193C159F1F2EC01F0ECD793C1B7
:1042000057F175EC01F001010B0E9A6F020E976FDA
:10421000070E0101995D18E099C1D7F116D8000980
:104220000FE00B0E01019A5D02E0050E04D0020EB4
:10423000995D02E1010E976F070E996F986B010C63
:104240000B0E01019A5DB3E1010C0101D751050A82
:1042500051E0060A4DE0070A34E0060A30E0030A9E
:1042600018E0010A51E192819293010E9A6F090EB2
:10427000E66EE66AC8C1E6FFC9C1E6FF9B0EE66EC0
:10428000010EE66E2EEC31F0106E060EE15E10505F
:10429000010C92A112D0C8C16FF3C9C170F3030120
:1042A0009B0E6D6F010E6E6F5EEC2FF0000904E047
:1042B00001019283020E29D00101060E26D087EF5C
:1042C00021F0D0C1E6FFD1C1E6FF5EEC2BF0E55254
:1042D000E552F3CF96F1D2C1E6FFD3C1E6FF5EEC23
:1042E0002BF0E552E552F3CF95F101010A0E0DD006
:1042F000B0EF21F00A0E9A6FFE0E945D07E094C1B4
:1043000056F135EC01F0010C050E9A6F010C01011C
:104310009851030A18E0020A0FE0010A20E1020E98
:10432000985D02E141EC24F0FE0E0101945D06E08F
:1043300010D90101010E05D0FCD811E10101030ED5
:104340009A6F986F000CEFD80AE093C155F12CECEE
:1043500001F0000904E093C156F135EC01F0000CC6
:1043600001019851020A2EE0030A21E0010A53E1FB
:1043700092B302D0060E4DD0070E9A6F95C153F13D
:1043800096C154F19351220DF3CFE9FFF4CFEAFF28
:10439000000EE9260A0EEA22EE52E9CF51F1EACFE9
:1043A00052F1AAEC00F00101946F010E09D0C1D8BE
:1043B00032E0020131A12FD0F8EC23F00101020E0E
:1043C000986F000C94C169F144EC03F000091AE005
:1043D000B6D80101730E626F090E636F94C161F16B
:1043E000B9EC02F0000905E073C945F210EC24F0C5
:1043F000F0D70201376B68EC23F094C160F19BECBD
:1044000002F0000C96D807E1A4D80101FE0E946FCB
:10441000090E9A6F010C000C0901006B060EE76E85
:104420000019E8AE02D0E73402D0E750005D2CE27C
:10443000040EE66EE66A00C9E9FFEA6AE9BEEA68C8
:10444000D890E936EA36960EE926020EEA22EECF39
:1044500010F0EFCF11F0126A10C0E6FF11C0E6FFB6
:1044600012C0E6FFD8C1E6FFD9C1E6FF84EC30F008
:10447000136E070EE15E1350000903E109010051BC
:1044800012000901002BCAD7060C0901036BA40E08
:10449000006F010E016F58D8EF50200804E1002B87
:1044A000000E0123F8D700C9C6F101C9C7F1010107
:1044B000010ED46F49D8EFCF02F9EF5033E0090174
:1044C0000351010A16E0010A29E1200E025D03E012
:1044D0002C0E025D05E138D8EF6A010E036F1ED085
:1044E0000D0E025D03E00A0E025D18E12DD8EF6AA1
:1044F00015D0200E025D12E00101D451D42BE96EDB
:10450000EA6AD890E936EA36C60EE926010EEA22B2
:1045100000C9EEFF01C9EDFF0901036B002B000E7E
:104520000123C8D7120093C158F1D9EC01F000095A
:10453000120094C155F12CEC01F00009120064C383
:10454000D5F165C3D6F1120000C9E9FF01C9EAFF40
:0E455000120041EC24F094C156F135EF01F059
:02455E00020158
:10456000306B010E316F0301180E3D6F84EC2FF09C
:104570000901006B060E005D05E2005191D9EF6A5A
:10458000002BF8D7010C0901FE0E026F020131A1C8
:10459000FE0C0901016B060E015D0AE2015180D992
:1045A000EF50010B03E101C902F902D0012BF3D74F
:1045B000FE0E025D01E1FE0C450E036F046B056B00
:1045C00033C2E9FF34C2EAFFEF5001E1FF0C33C20E
:1045D000E6FF34C2E6FF5CEC31F0E552E552F3CF82
:1045E00033F2F4CF34F203C942F304C943F367D979
:1045F00004E00901FE0E026F5ED00EEC30F00901FE
:10460000006F00AF02D0026956D0016B0C0E015D45
:1046100021E20EEC30F00901006F01510201EA6A5B
:104620003325E96E3451EA22EF500901005D06E0BE
:10463000120E0327000E042305230CD0005108E1BD
:104640000901012B0C0E015D05E20EEC30F0F8D7EC
:10465000012BDCD70C0E015D2BE10251080DF3CFCD
:1046600006F9F4CF07F9000E0627020E072333D907
:10467000010EEF6E30D9EB6A020EEB6A0EEC30F0F1
:10468000E66E29D9030E03D9030E2AD9010EFFD8ED
:10469000030E26D9020EFBD8060EF9D8060E20D935
:1046A000010E1ED9E552E750EF6E0201302B03D008
:1046B00018EC30F098D718EC30F0090102511200D4
:1046C00036C237F205D802013651EAD8EF6A120035
:1046D00002013751080DF3CFAFF9F4CFB0F9000E56
:1046E0000901AF27020EB023F1D8EF50020B03E00F
:1046F00018EC30F00DD0EAD8EF50040B09E004ECD0
:1047000030F00301A00E4B6F53EC30F00009F9E1DB
:10471000F90EDCD8E850EF160201319312000201C5
:104720003851080DF3CF01F9F4CF02F9000E090159
:104730000127020E02239F0E106EBCD8E850EF1620
:10474000B9D8EF50010B25E0B5D8EF50020B24E1AA
:10475000020131B31ED0AED8EE52EECF13F0EFCF40
:1047600014F0156AA7D8030EBBD8EE501324106EB0
:10477000EE501420116EEE501520126E10C042F350
:1047800011C043F39CD805E195D8EF820201318333
:1047900003D090D8EF8A000C0EEC30F00901006FC6
:1047A00089D8EE52EE2A000EED22EECF10F0EDCFBA
:1047B00011F080D8060E94D8EECF12F0EFCF13F0A0
:1047C00000011250101805E11350111802E172D8BF
:1047D000EF8C090100511200010C010C12001200B3
:1047E000F36AF46A1200056A066A076A1200000C8E
:1047F000020131A1000C0901AF6B060EAF5D08E2AA
:10480000AF514ED8EF50010B01E0000CAF2BF5D7A4
:104810000201010E006F400E036F046B056B010C6B
:104820000901000EB16F020EB26F020100A506D0A1
:10483000400E325D03E30201376B4ADF020100B52F
:1048400015D031A302D0008B000C03C23FF304C289
:1048500040F30301A00E3E6F8DEC2FF0000905E13F
:10486000020100853183326B01D0000C45C244F354
:10487000F0EC2FF00201322B032B000E0423052352
:10488000010C0201376B24DF0201006B010C28D8F8
:10489000E552E750EF6E0EEC30F0E66E6BEF24F071
:1048A000080DF3CFE9FFF4CFEAFF000EE926020E70
:1048B000EA22120001C9E9FF02C9EAFF120003015E
:1048C000A00E416FC3EC2FF000091200AFC9E9FF41
:1048D000B0C9EAFF120006C9E9FF07C9EAFF1200E2
:0848E000E926000EEA22120095
:0848E800D9C2F3FFD8C2F4FFAE
:1048F0001200DAC201F9DBC202F9DCC203F9DDC23F
:1049000004F90901010E056F090E066F05C9E9FFDB
:10491000EA6E030E9AD9EF50E66E030E90D900C9E5
:10492000EFFF84D9020E91D9010E85D9EF50E66EC2
:104930007DD9020E84D9010E7ED900C9EFFF01C9CD
:1049400004F002C905F003C906F004C907F012001B
:104950000901406B416B426B436BDEC23EF9DFC223
:104960003FF9E0C23CF9E1C23DF9D8903D333C3318
:104970003CC910F03DC911F03C07000E3D5B1050E2
:10498000111018E03EC9E9FF3FC9EAFF020E3E27B9
:10499000000E3F23EECF10F0EFCF11F000011050CA
:1049A000090140270001115009014123000E422353
:1049B0004323DED70201E051010B0EE03EC9E9FFBF
:1049C0003FC9EAFFEFCF10F0000110500901402766
:1049D000000E41234223432309014251431109E0C0
:1049E00040514225406F41514321416F426B436B1F
:1049F000F3D740C910F041C911F0101E111E10C0AC
:104A0000F3FF11C0F4FF12000901010E006F016BEA
:104A1000026B0201E251E3114EE0400EE25D000E36
:104A2000E35904E3400E106E116A04D0E2C210F0A4
:104A3000E3C211F010C005F9090110500201576FCF
:104A4000586B0201060E556F090E566F20EC15F0DB
:104A500009010551106E116A10500201E25F1150F8
:104A6000E35B0901046B0551045DD3E20451EA6A7A
:104A7000060FE96E090EEA22EFCF03F900510AE1B1
:104A800003510125016F0351015D0DE2022B0BE182
:104A9000012B09D003510225026F0351025D03E28D
:104AA000012B01E1022B005102E0000E01D0010EAA
:104AB000006F042BD8D70901021D026F011DF36E90
:104AC00002C9F4FF12000201E451390805E3300E77
:104AD000E45D02E3300E0FD0E451460805E3410ED9
:104AE000E45D02E3370E07D0E451660806E3610E89
:104AF000E45D03E3570EE45D1200FF0C010E0201BA
:104B0000EA6AE525E96EE651EA22EFCFE4F2DBDF5F
:104B10000901236FE5C2E9FFE6C2EAFFEFCFE4F245
:104B2000D2DF0901246FFF0E235D03E0FF0E245D39
:104B300001E1000C2439F00B2311E7C2E9FFE8C2C0
:104B4000EAFFEF6E010C0901236BA6B2FED72F0E10
:104B5000A616A6840201EBC2E9FFECC2EAFFEB2B2A
:104B6000000EEC23EF50A86E0901232B0201ED513A
:104B70000901D880235501E2A86AEAC210F0116A3F
:104B80001050AA6E0201E9C210F0EAC211F0E92B3E
:104B9000000EEA231050A96E550EA76EAA0EA76E3E
:104BA000A6820000A6B2FED7A850D4E1A6940901BF
:104BB000235100D01200F1C210F01050AA6EF0C2C2
:104BC000A9FF3F0EA6160201EEC2E9FFEFC2EAFFFF
:104BD000EE2B000EEF23EFCF1CF9A680A8500901A1
:104BE0001C5D01E0010C1C5101E1000CA92AEBE164
:104BF000AA2AE9D7F2C202F9F3C203F90901006B4C
:104C0000016B0201F4510901005D0201F551090136
:104C100001590BE202C9E9FF03C9EAFF022B000EAA
:104C20000323EF6A002B0123ECD7120005C9E9FF2B
:104C300006C9EAFF1200E926000EEA221200FBDF95
:104C4000E552E750EF6E16EF26F0F5DFEFCF00F9F3
:044C500016EF26F045
:0C4C5400140E0201576F586B0201080E8D
:104C6000556F090E566F20EC15F0F00E090108156E
:104C7000400801E0A1D00F0E0815040DF350106E8E
:104C8000116A140E105E000E115A10C01CF910505B
:104C9000140801E291D01C5100080BE21C510201E2
:104CA000576F586B02011D0E556F090E566F20ECA1
:104CB00015F012C900F913C901F90901126B136B40
:104CC000140E16D9080EDE6F090EDF6FA8EC24F063
:104CD000F3CF04F9F4CF05F90901041F051F1C5196
:104CE000000810E21C5104D91D0EDE6F090EDF6FA3
:104CF000A8EC24F0F3CF06F9F4CF07F90901061F59
:104D0000071F02D0066B076B040EF2D8040EDE6F8D
:104D1000090EDF6FA8EC24F0F3CF02F9F4CF03F90A
:104D20000301080E596F090E5A6FB5D809010251D7
:104D3000001942E1035101193FE1F00E0815400846
:104D40003BE103014C514D110CE04CC3E9FF4DC355
:104D5000EAFF18C9EEFF19C9EEFF1AC9EEFF1BC919
:104D6000EEFF4EC3E9FF4FC3EAFF060EDBD814C9BE
:104D7000EEFF15C9EEFF16C9EEFF17C9EEFF50C3CF
:104D8000E9FF51C3EAFF11C9EFFF09011C51126E7F
:104D9000136A12500A5D106E13500B59116E140EE7
:104DA000105E000E115A52C3E9FF53C3EAFF10C050
:104DB000EEFF11C0EDFF010C7AEC15F0000C0901BB
:104DC000450E286F296B140E0301572509012A6F20
:104DD000000E0301582109012B6F0101FD2B000E6C
:104DE000FE23FDC12CF9FEC12DF909012E6B400EE9
:104DF0002F6F640E306F56C331F9326B336BB8C20C
:104E000034F9B9C235F9BAC236F9BBC237F954C35D
:104E1000E9FF55C3EAFF060E85D8EECF38F9EECF8D
:104E200039F9EECF3AF9EFCF3BF90301280E596F6C
:104E3000090E5A6F30D8140E5BD8280EDE6F090E9B
:104E4000DF6FA8EC24F0F3CF32F9F4CF33F9140E6E
:104E5000030157250201626F000E03015821020170
:104E6000636F0201616B54C3E9FF55C3EAFF54C38A
:104E70005FF255C360F272EC16F0140E0201536F2C
:104E8000546B0201280E516F090E526F64EC14F03E
:104E9000F36AF46A120027D8020E35D8020E38D809
:104EA000020E2BD8020E39D8040E2DD8040E30D89D
:104EB000040E23D8040E31D8060E25D8060E28D8A5
:104EC000060E1BD8060E29D80A0E1DD80A0E20D8A9
:104ED0000A0E13D80A0E03D83CC9EFFF120022D8DD
:104EE000010E92EF27F059C3E9FF5AC3EAFF1200FF
:104EF0000201E06FE16B0201120014D8E552E750A5
:104F0000EF6E73EF27F00ED8EFCF3CF973EF27F079
:104F1000E6DFEF50E66E73EF27F0E1DF3CC9EFFF0D
:0C4F200073EF27F0E926000EEA221200D1
:044F2C004854545041
:104F30002F312E3020353033200D0A0D0A53657283
:104F40007669636520556E617661696C61626C6536
:104F50000D0A000D0A0D0A00485454502F312E300E
:104F600020323030204F4B0D0A436F6E74656E74E3
:104F70002D747970653A2000485454502F312E30EA
:104F800020343034204E6F7420666F756E640D0AC5
:104F90000D0A4E6F7420666F756E642E0D0A0061E7
:104FA0007564696F2F782D77617665006170706C1C
:104FB00069636174696F6E2F6A6176612D617263D6
:104FC0006869766500696D6167652F6A706567005D
:104FD000696D6167652F67696600746578742F6A0B
:104FE00061766173637269707400746578742F639D
:104FF0007373006170706C69636174696F6E2F6A9E
:105000006176612D766D00746578742F68746D6CAF
:1050100000746578742F706C61696E0047756573F4
:1050200074004E6F00537570657220557365720081
:105030000D0A4E6F772072756E6E696E6720617013
:10504000706C69636174696F6E2E2E2E000D0A52AA
:105050006561647920746F20646F776E6C6F616432
:105060002046696C652053797374656D20496D61C4
:105070006765202D2055736520586D6F64656D2020
:1050800070726F746F636F6C2E0D0A000D0A4448C6
:105090004350202620495020476C65616E696E6739
:1050A0002064697361626C65642E0D0A000D0A4408
:1050B000484350202620495020476C65616E696E38
:1050C0006720656E61626C65642E0D0A000D0A44EE
:1050D000656661756C74205375626E6574204D61F0
:1050E000736B2028000D0A44656661756C74204757
:1050F00061746577617920416464726573732028F7
:10510000000D0A44656661756C7420495020416445
:1051100064726573732028000D0A53657269616CAF
:10512000204E756D626572202800323030206F6B22
:105130000D0A00323236205472616E736665722039
:10514000436F6D706C6574650D0A00313235204413
:105150006F6E652E0D0A00313530205472616E730A
:1051600066657272696E6720646174612E2E2E0D01
:105170000A00353330204C6F67696E207265717597
:10518000697265640D0A00353032204E6F742069F3
:105190006D706C656D656E7465640D0A0035303038
:1051A000200D0A00323231204279650D0A00323377
:1051B00030204C6F6767656420696E0D0A003333D9
:1051C000312050617373776F7264207265717569F5
:1051D0007265640D0A003232302052656164790DC7
:1051E0000A0041424F5200504F52540053544F5204
:1051F00000515549540050415353005553455200F6
:105200001C0E0201576F586B0201000E556F090EFC
:10521000566F20EC15F07AEC15F00301000E626F6A
:10522000090E636FF5D80901010E001912E1015151
:1052300010E10451106E116A060E10180AE11150A7
:1052400008E10551126E136A040E121801E11350A1
:1052500001E0000C020E061905E1075103E106D931
:10526000EF6A0DD0010E061906E1075104E1010EA7
:10527000FDD8EF6E04D0020EF9D8EF6E000C0201DB
:10528000B8510901185D2EE10201B9510901195DFA
:1052900029E10201BA5109011A5D24E10201BB5161
:1052A00009011B5D1FE15BC3E9FF5CC3EAFF08C99D
:1052B000EEFF09C9EEFF0AC9EEFF0BC9EEFF0CC9EC
:1052C000EEFF0DC9EEFF5BC3E9FF5CC3EAFF060E0C
:1052D000D7D80EC9EEFF0FC9EEFF10C9EEFF11C9F6
:1052E000EEFF010C000C010E0901006F016B026B57
:1052F000080E036F060E046F040E056F03016105AF
:105300000BE1010E0901066F076B1269136914693D
:1053100015691669176914D0020E0901066F076B2B
:105320005FC3E9FF60C3EAFFEECF12F9EECF13F9D6
:10533000EECF14F9EECF15F9EECF16F9EFCF17F93E
:10534000BCC208F9BDC209F9BEC20AF9BFC20BF955
:10535000C0C20CF9C1C20DF9B8C20EF9B9C20FF939
:10536000BAC210F9BBC211F97AD8EF500E19020176
:10537000C2151BE174D8010E83D8EF5009010F1933
:105380000201C31512E16BD8020E7AD8EF50090161
:1053900010190201C41509E162D8030E71D8EF504B
:1053A000090111190201C51509E0C6C218F9C7C2E1
:1053B00019F9C8C21AF9C9C21BF909D050D8EECFE1
:1053C00018F9EECF19F9EECF1AF9EFCF1BF9030157
:1053D000000E626F090E636F1BD81C0E0201626F14
:1053E000636B0201060E616F0201120E5F6F090E00
:1053F000606F72EC16F01C0E0201536F546B0201C9
:10540000000E516F090E526F64EC14F0C9EF16F0E4
:1054100032D819D8F3CFEEFF11C0EDFF2CD8020E11
:105420002FD811D8020EF3CFEBFF030E11C0EBFF04
:1054300022D8060E25D807D8060EF3CFEBFF070EAD
:1054400011C0EBFF1200EECFD8F2EDCFD9F274EC21
:1054500024F0F3CF10F0F4CF11F03BEF2AF05FC34C
:10546000E9FF60C3EAFF060E40EF2AF05DC3E9FFE3
:105470005EC3EAFF120062C3E9FF63C3EAFF1200E2
:08548000E926000EEA221200E9
:085488000B01BD6BBE8171EC4C
:1054900013F0F7EC32F0ADEC17F03AEF00F0090141
:1054A000010EB46F0901B45101E1FDD0B46B0B01E1
:1054B000BD51040A01E1D7D0070A01E1A1D0050AD4
:1054C00001E187D0010A72E0050A3FE0070A36E0F1
:1054D000050A02E0010AE6E10201B30E5D6F090E62
:1054E0005E6F0201BF0E5B6F0B0E5C6FBFEC15F0C1
:1054F000000915E10201160ED66F8FEC31F0010B99
:10550000D1E0B1EC15F00009CDE10201B86BB96B47
:10551000BA6BBB6B0B01BE810CEC1BF0C3D709014E
:10552000010EB46FB35103E10B01020E39D0060E28
:10553000B35D01E095D00B01050E32D00901B46BCB
:1055400004EC33F00009AEE0ABD00301C90E526F9A
:105550000B0E536F0301B30E506F090E516F030111
:10556000BF0E4E6F0B0E4F6F0301AF0E4C6F090E47
:105570004D6F2AEC26F0000916E00901010EB46F08
:10558000B30503E10B01030E0BD0060EB35D03E17F
:105590000B01060E05D0110EB35D04E10B01070EE1
:1055A000BD6F80D7B46B7AEC15F07AD0C9CB41F1DE
:1055B000CACB42F10101AF0E3F6F090E406F0101EE
:1055C000BF0E3D6F0B0E3E6F3DEC19F0000915E06C
:1055D00012D0C9CB6EF1CACB6FF10101AF0E6C6F67
:1055E000090E6D6F0101BF0E6A6F0B0E6B6F2DEC14
:1055F00004F0000902E00B01BD6B0901B46B52D746
:10560000BD6B290ED880C955000ECA5529E3030188
:10561000ED0E1F6F0B0E206F0301EB0E1D6F0B0EB7
:105620001E6F0301C90E1B6F0B0E1C6F0301CB0E07
:10563000196F0B0E1A6F0301B30E176F090E186F57
:105640006DEC2CF000090AE0080E0901B35D06E1DB
:10565000010EB46F0B01040EBD6F02D00B01BD6BC8
:105660007AEC15F01FD734EC14F0000901E11AD7D9
:10567000EDCB29F3EECB2AF3EBCB27F3ECCB28F3DE
:10568000C9CB26F30301CB0E246F0B0E256F03014C
:10569000236B0301BF0E216F0B0E226FE7EC2CF082
:1056A0000B01BD6BFFD651EC03F01AEC1BF00301AC
:0C56B00077A102D00B01BE911EEF14F098
:0456BC00FF0EE3CF2B
:1056C000EAFFE552FF0EE3CFE9FFE552E66AE66A3C
:1056D000D9CFE6FFDACFE6FFFC0EE124D96EFF0E4C
:1056E000E220DA6EE66AE66AE66A200EEF5C06E021
:1056F000090EEF5C03E0EF6603D03FD0EE50F5D724
:105700002D0EEF5C03E1FF0EE32A03D02B0EEF5CBE
:1057100001E1EE502F0EEF6424D03A0EEF6021D05D
:10572000D890F90EE336FA0EE336FD0EDECFE3FF36
:10573000FE0EDDCFE3FFD890F90EE336FA0EE33626
:10574000D890F90EE336FA0EE336FD0EE350DE266E
:10575000FE0EE350DD22300EEE5CDE26000EDD2272
:10576000D9D7FF0EE3CFE8FFE85207E0F90EE31EBA
:10577000E32AFA0ED8B4E306E31EE552E552E552F9
:10578000FF0EE3CFDAFFE552FF0EE3CFD9FFE5527C
:10579000E1CFE9FFE2CFEAFFED52ED52EECFF3FFAA
:1057A000EFCFF4FF1200D9CFE6FFDACFE6FFFA0E13
:1057B000E3CFD9FFFB0EE3CFDAFFFD0EE35209E79B
:1057C0002D0EDE6EFC0EE31EE32AFD0ED8B4E306BA
:1057D000E31EE652E652E652FD0EE124E76EFF0EAE
:1057E000E220E46EE652F70EE3CFE6FFF70EE3CFDA
:1057F000E6FF43EC2CF0F90EE124E96EFF0EE22007
:10580000EA6E33EC2CF00AE130EC2CF009E133ECD9
:105810002CF008E130EC2CF007E108D03EEC2CF045
:1058200039EC2CF03EEC2CF039EC2CF03EEC2CF06A
:10583000DE6AF90EE126FF0EE222FF0EE3CFDAFF69
:10584000E552FF0EE3CFD9FFE552FC0EE124E96EED
:10585000FF0EE220EA6EEECFF3FFEFCFF4FF12006F
:10586000EF380F0B1200EF500F0B02E1EE52D8840D
:105870001200EF380F0B300FDE6E1200EE500F0BE0
:10588000300FDE6E1200FC0EE3CFE9FFFD0EE3CF1A
:10589000EAFF100EE66EEE6AEE6AEF6AD890FD0E31
:1058A000E336FE0EE336ED36ED36EF36FF0EE30659
:1058B00009E064EC2CF0EE5264EC2CF0EE5264EC57
:1058C0002CF0EDD7E56E1200030EEF24E8B6EF6E74
:0A58D000300EEF24E8BEEF6E000C6E
:0658DA00080E0201576FE9
:1058E000586B0201000E556F090E566F20EC15F033
:1058F00002C92EF903C92FF90901026B036B080EC7
:105900000201E06FE16B0201000EDE6F090EDF6F36
:10591000A8EC24F0F3CF28F9F4CF29F90901281FC6
:10592000291F080E106ED9D8E850EF5ED6D8EF5078
:105930000201576F586B19C355F21AC356F220EC87
:1059400015F0CBD8EF500201E06FE16B19C3DEF226
:105950001AC3DFF2A8EC24F0F3CF2AF9F4CF2BF925
:1059600009012A1F2B1F040E0201E06FE16B0201E7
:10597000280EDE6F090EDF6FA8EC24F0F3CF2CF9B0
:10598000F4CF2DF90301000E2B6F090E2C6F7AD87E
:1059900017C3E9FF18C3EAFF00C9EFFF1DC3E9FF02
:1059A0001EC3EAFF04C9EEFF05C9EDFF1FC3E9FFEF
:1059B00020C3EAFF06C9EEFF07C9EDFF09012E511A
:1059C0002C1902E12F512D1901E0000C010C0901E5
:1059D000016B23C300F9026B036B27C304F928C3CF
:1059E00005F929C306F92AC307F903012651E66E12
:1059F000E66A24C3E6FF25C3E6FF080EE66E090E3D
:105A0000E66EA3EC30F0106E060EE15E105003015E
:105A1000000E2B6F090E2C6F35D8080E03012625BA
:105A20000201E06FE16B000EE1230201000EDE6F68
:105A3000090EDF6FA8EC24F0F3CF02F9F4CF03F9DD
:105A4000080E030126250301576F586B000E5823DB
:105A50000301010E566F21C354F322C355F3DFEC4B
:105A600026F0080E030126250201536F546B000E29
:105A700054230201000E516F090E526F64EC14F0B2
:105A8000C9EF16F02FD8040E15D8040EF3CFEBFF94
:105A9000050E1FD8060E0ED8060EF3CFEBFF070E2D
:105AA00018D8020E07D8020EF3CFEBFF030E11C079
:105AB000EBFF1200E926000EEA22EECFD8F2EDCF7E
:105AC000D9F274EC24F0F3CF10F0F4CF11F072EFB0
:105AD0002DF011C0EBFF72EF2DF01BC3E9FF1CC3CB
:0E5AE000EAFF12002BC3E9FF2CC3EAFF1200FD
:025AEE004D6FFA
:105AF0006474726F6E6978205443502F495020535C
:105B00007461636B2056332E3033000D0A5072657A
:105B1000737320616E79206B657920666F72204304
:105B20006F6E66696775726174696F6E206D656E00
:105B3000752E00444843502F476C65616E696E674F
:105B40002E2E2E000D0A0D0A0D4D785765625372E8
:105B500076722044656D6F204170706C696361746A
:105B6000696F6E2076312E3020284D6F6474726F0D
:105B70006E6978205443502F495020537461636BF1
:105B80002056332E30332C204D6172203036203297
:105B9000303036290D0A0D0A09313A204368616E0A
:105BA000676520426F6172642073657269616C2061
:105BB0006E756D6265722E0D0A09323A2043686176
:105BC0006E67652064656661756C7420495020615C
:105BD0006464726573732E0D0A09333A2043686159
:105BE0006E67652064656661756C742067617465B5
:105BF00077617920616464726573732E0D0A0934CC
:105C00003A204368616E67652064656661756C74EF
:105C1000207375626E6574206D61736B2E0D0A09B9
:105C2000353A20456E61626C652044484350202619
:105C300020495020476C65616E696E672E0D0A0918
:105C4000363A2044697361626C65204448435020B1
:105C50002620495020476C65616E696E672E0D0ADB
:105C600009373A20446F776E6C6F61642046696C27
:105C7000652053797374656D20496D6167652E0DDC
:105C80000A09383A205361766520262051756974D7
:105C90002E0D0A0D0A456E7465722061206D656EC9
:105CA000752063686F6963652028312D38293A2093
:105CB000000D0A496E76616C696420696E707574B6
:105CC000207265636569766564202D20496E707564
:105CD000742069676E6F7265642E0D0A5072657369
:105CE0007320616E79206B657920746F20636F6E0D
:105CF00074696E75652E2E2E0D0A001B5B324A00EC
:105D0000DACFE4FFE2CFDAFFE9CFE4FFEACFE4FF46
:105D1000F6CFE4FFF7CFE4FFF5CFE4FFF3CFE4FFE6
:105D2000F4CFE4FFFACFE4FF00EE00F0100EE80439
:105D300003E3EECFE4FFFBD700EE10F0080EE8041B
:105D400003E3EECFE4FFFBD7E652F2A414D09E0E9D
:105D5000D76E580ED66E0301642B000E65236623A2
:105D6000672303016A0706E1640E6A6F0301682B6B
:105D7000000E6923F2949E50200B05E09D50200BED
:105D800002E049EC32F09E50100B05E09D50100BE4
:105D900002E05FEC32F0E55200EE17F0080EE80486
:105DA00003E3E5CFEDFFFBD700EE0FF0100EE804A4
:105DB00003E3E5CFEDFFFBD7E5CFFAFFE5CFF4FF37
:105DC000E5CFF3FFE5CFF5FFE5CFF7FFE5CFF6FF32
:105DD000E5CFEAFFE5CFE9FFE5CFDAFF110088D88C
:105DE000ADEC34F0AFEC22F0F3EC0EF035EC32F029
:105DF00071EC31F0ADEC31F03EEC32F0FCEC31F016
:105E000013EC32F028EC32F00201140ED66F8FEC56
:105E100031F00001F36FE0EC1DF044EC2AF05EEC91
:105E20000AF05CEC20F00201160ED66F8FEC31F018
:105E3000010B06E10001010EFE6F0301070E756FF5
:105E40000201150ED66F8FEC31F0020B0CE0000151
:105E5000FF510301645D106E320E105C04E364C3F5
:105E6000FFF0939C8A7C4FEC2AF0FEEC0AF06BEC7E
:105E700020F008D80001FE510301785DE1E078C30D
:105E8000FEF0DED703016C2B0C0E6C5D01E36C6B36
:105E9000C11C0F0B6C5D0FE2C30EC2166C51040DDA
:105EA000F350C212C280C282C2B2FED7030125D80B
:105EB000C4CFEFFF120021D8EF6A1200350E0201A5
:105EC000F06FF16B6DC3EEF26EC3EFF2DBEC25F019
:105ED00000090DE13E0E0201F06FF16B6FC3EEF2AF
:105EE00070C3EFF2DBEC25F0000901E1010C000CBE
:105EF000F18ED56AF28EF28C12006C51EA6ACA0FEA
:085F0000E96E020EEA22120014
:085F08003DC373F30301726B4A
:105F10000301080E716F65EF34F03FC3AFF940C362
:105F2000B0F9C750040B01E0010EE5D8FAE1C580D5
:105F3000C5B0FED7A1B6010C3EC374F3E1D801E0B1
:105F4000010CC750040B01E0010ED5D8FAE1C5BC25
:105F500019D0B0C974F3D4D801E0010CC750040BB8
:105F600001E0010EC8D8FAE1AFC974F3C9D801E065
:105F7000010CC750040B01E0010EBDD8FAE1C5AC1D
:105F8000000C020C020C42C33FF343C340F341C375
:105F90003EF3C3DF0901086FE85005E178D8090135
:105FA000086FE85002E008511200C750040B01E0EE
:105FB000010EA1D8FAE1C580C5B0FED7A1B6010C8B
:105FC000030141290301746F9BD801E0010CC75004
:105FD000040B01E0010E8FD8FAE1C5AC000C020CF5
:105FE000C750040B01E0010E86D8FAE144C374F3F4
:105FF00087D801E0010CC750040B01E0010E7BD8EB
:10600000FAE1C5AC000C020CC750040B01E0010E14
:1060100072D8FAE1C584C5B4FED7000C74EC34F034
:10602000C5B6FED7C59AC588C5B8FED7C9501200F7
:1060300074EC34F0C5B6FED7C58AC588C5B8FED79E
:10604000C584C5B4FED7000C46C342F347C343F32F
:1060500045C341F398DF0901006FE85016E10301E1
:106060004A514A0700090EE0D9DFE66E030148C332
:10607000E9FF49C3EAFF482B000E4923E552E750E8
:10608000EF6EEDD7D5DF0901006F00511200C75048
:10609000040B01E0010E2FD8FAE1C584C5B4FED788
:1060A000A1B6010C000CC750040B01E0010E23D86F
:1060B000FAE1C580C5B0FED7A1B6010C4BC374F39D
:1060C0001FD801E0010CC750040B01E0010E13D8EA
:1060D000FAE1A1B6010CC5BC03D00901B36B03D032
:1060E0000901040EB36FC584C5B4FED7A1B6010C77
:1060F0000901B3511200106E1F0EC51410101200CA
:0861000079EC34F000091200F3
:08610800FB0EE3CFF6FFFC0ED5
:10611000E3CFF7FFFD0EE3CFF8FFFE0EE3CFE9FF7D
:10612000FF0EE3CFEAFFF90EE35003E1FA0EE3506E
:1061300009E0F90EE30602E2FA0EE3060900F55063
:10614000EE5CF1E01200D9CFE6FFDACFE6FFFA0EFF
:10615000E3CFD9FFFB0EE3CFDAFFFC0EE3CFE9FF7D
:10616000FD0EE3CFEAFFE9CFF3FFEACFF4FFF80E2D
:10617000E35003E1F90EE35008E0F80EE30602E213
:10618000F90EE306DECFEEFFF2D7FF0EE3CFDAFF24
:10619000E552FF0EE3CFD9FFE5521200FB0EE3CF2D
:1061A000F6FFFC0EE3CFF7FFFD0EE3CFF8FFFE0E88
:1061B000E3CFE9FFFF0EE3CFEAFFE9CFF3FFEACF3A
:1061C000F4FFF90EE35003E1FA0EE35009E0F90E93
:1061D000E30602E2FA0EE3060900F5CFEEFFF1D77F
:1061E0001200FB0EE3CFF6FFFC0EE3CFF7FFFD0E30
:1061F000E3CFF8FFFE0EE3CFE9FFFF0EE3CFEAFFA8
:106200000900F550EF5C02E1EE66FAD71200FB0ED2
:10621000E3CFF6FFFC0EE3CFF7FFFD0EE3CFF8FF71
:10622000FE0EE3CFE9FFFF0EE3CFEAFFE9CFF3FF76
:10623000EACFF4FF0900F5CFEFFFEE66FBD71200BF
:10624000FE0EE3CFE9FFFF0EE3CFEAFFF36AF46A45
:10625000EE5203E0F34AF42AFBD71200D9CFE6FF4F
:10626000DACFE6FFFA0EE3CFD9FFFB0EE3CFDAFF7A
:10627000FC0EE3CFE9FFFD0EE3CFEAFFE9CFF3FF2A
:10628000EACFF4FFF80EE35003E1F90EE3500BE020
:10629000F80EE30602E2F90EE306DECFEFFFEE664C
:1062A000F1D7DD52EFD7FF0EE3CFDAFFE552FF0E55
:1062B000E3CFD9FFE5521200FE0EE3CFE9FFFF0E58
:1062C000E3CFEAFFE9CFF3FFEACFF4FF610EEF5C23
:1062D00005E67B0EEF5C02E7DF0EEF16EE52F6E10D
:0262E0001200AA
:0E62E200AA6AA96A3F0EA6160901B80E006F3F
:1062F000020E016FA950106E116A120E105C000E92
:1063000011580CE2A68000C9E9FF01C9EAFF002B81
:10631000000E0123A8CFEFFFA92AECD71200D6C2A6
:10632000A9FFAA6AA6B2FED73F0EA616A680A8505D
:106330001200D7C2A9FFAA6AA6B2FED72F0EA616D0
:10634000A684550EA76EAA0EA76EA6820000A6B25E
:10635000FED7A69400D012001200240EAC6E900E50
:10636000AB6E080E7E6E02011F0E7CD8080A36E066
:106370000F0A32E0010A2AE0030A23E0010A1CE0C6
:10638000070A15E0010A0EE0030A07E0010A28E106
:106390000901340E1C6F820E1DD009018C0E1C6F7A
:1063A000200E18D00901450E1C6F100E13D00901E4
:1063B000220E1C6F080E0ED00901100E1C6F040E69
:1063C00009D00901080E1C6F020E04D00901030E4A
:1063D0001C6F010E1D6F08D0AC0E03D0560E01D0FD
:1063E000AC0E09011C6F1D6B1CC9AFFF1DC910F05D
:1063F000116A10507F6E12000201230E33D8926E84
:106400000201240E2FD8936E0201250E2BD8D80935
:10641000946E0201280E26D8976E0201290E22D80A
:106420001009986E120002012A0E1CD8896E020112
:106430002B0E18D88A6E02012C0E14D88B6E020116
:106440002F0E10D88E6E0201300E0CD88F6E1200F7
:106450000201310E07D8C16E0201320E03D87F0B44
:0A646000C06E1200D66F8FEF31F00E
:06646A000001EC6BE06B89
:10647000E16BEA6BEB6B9D9A9D9812009D8A9D984B
:1064800012000001E16BE1C0E0F0EB6BEBC0EAF061
:106490001200060EAB1402E0AB98AB889EAA0ED099
:1064A0000001EB51EA6AE20FE96E000EEA22AECF7C
:1064B000EFFFEB2B070EEB15EB6FF0D7120000018F
:1064C000E051E15D0DE0E051EA6A600FE96E000E17
:1064D000EA22EF50AD6EE02B7F0EE015E06F120068
:1064E0009D98120012000001EC5112000001EA51C7
:1064F000EA6AE20FE96E000EEA22EFCFAFF9EA2B6B
:10650000070EEA15EA6F0901AF5112000001E129F7
:10651000106E116A7F0E1016000E11160001E05168
:10652000126E136A1250101802E11350111802E192
:106530000400ECD7F29E9DB805D0EDC0ADFF9D885C
:10654000F28E11D00001E151EA6A600FE96E000E8F
:10655000EA22EDC0EFFF0001E12B7F0E0001E11503
:106560000001E16FF28E12000001EE519F0805E27A
:10657000EE390F0B0F0B570F04D0EE390F0B0F0B2B
:10658000300F0001ED6FC2DF0F0E0001EE1509089C
:1065900004E20F0EEE15570F03D00F0EEE15300F5D
:1065A0000001ED6F86EF32F00001EFC0E9FFF0C0AF
:1065B000EAFFEF2B000EF023EFCF08F9EF5004E0D5
:1065C00008C9EDF0A3DFF0D712000001F1C0F6FF1B
:1065D000F2C0F7FFF12B000EF2230800F5CF00F90F
:0E65E000F55004E000C9EDF091DFEFD7120096
:0265EE000B019F
:1065F000EF6BF069F169F269F369F469F569F66BBB
:10660000F76BF86BF96B12000B01EF5129E10301F5
:10661000260E5D6F090E5E6F03011C0E5B6F090E87
:106620005C6F00EC29F000092CE00901265115E10E
:106630001CC9F0FB1DC9F1FB1EC9F2FB1FC9F3FB0E
:1066400020C9F4FB21C9F5FB22C9F6FB23C9F7FBDE
:1066500024C9F8FB25C9F9FB010C0B01010EEF6FF2
:1066600034EC14F000090CE00301616B03011C0E13
:106670005F6F090E606F73EC29F00B01EF6B010C7B
:10668000000C010CFACBE9FFFBCBEAFFEECF22F9BD
:10669000EECF23F9EECF24F9EFCF25F90301010E58
:1066A000616F03011C0E5F6F090E606F73EF29F0BD
:1066B000FCCBE9FFFDCBEAFF0B01F651EE1808E138
:1066C000F751EE1805E1F851EE1802E1F951EE1814
:1066D00014E00201C6510B01F65D20E10201C75131
:1066E0000B01F75D1BE10201C8510B01F85D16E1DA
:1066F0000201C9510B01F95D11E1FECBE9FFFFCBAE
:10670000EAFFF0CBEEFFF1CBEEFFF2CBEEFFF3CBE7
:0E671000EEFFF4CBEEFFF5CBEEFF010C000C1C
:02671E005458CD
:10672000540048544D00434C4100435353004A53D6
:10673000000047494600434749004A5047004A4144
:10674000520057415600545854005A5458005A4861
:1067500054005A434C005A4353005A4A5300485479
:1067600054502F312E3020323030204F4B00436FA9
:106770006E74656E742D747970653A2000436F6E87
:1067800074656E742D456E636F64696E673A206739
:106790007A69700D0A00457870697265733A203025
:1067A0000D0A0043616368652D436F6E74726F6CF0
:1067B0003A206D61782D6167653D3330302C206D56
:1067C0007573742D726576616C69646174650D0A08
:1067D0000047455400494E4445582E48544D004CFE
:0967E0004F47494E2E4347490082
:0667EA002A0EF66E000EFF
:1067F000F76E000EF86E02010900F550FB6F0900FC
:10680000F550FC6F03E1FB6701D03DD00900F55066
:10681000F66F0900F550F76F0900F550F86F0900A1
:106820000900F550E96E0900F550EA6E090009000B
:106830000900F550F96F0900F550FA6F09000900D9
:10684000F6CFFDF2F7CFFEF2F8CFFFF2F6C2F6FF79
:10685000F7C2F7FFF8C2F8FF0201F95302E1FA5359
:1068600007E00900F550EE6EF907F8E2FA07F9D7EC
:10687000FDC2F6FFFEC2F7FFFFC2F8FF0201FB07F1
:08688000000EFC5BBFD7120003
:086888004E6F7420496D706C25
:10689000656D656E7465640073656C6563746564CD
:1068A00000636865636B65640064697361626C654D
:1068B00064003C212D2D002D2D3E006F6E006F6673
:0968C00066005570646174650006
:0668CA003F0EC716C66A6E
:1068D000C56A03017151C6127251C7129486948819
:1068E000C68A73C3C8FF1200C586C7A0FED7C950A9
:1068F000120074C3C9FFC6BEFF0CC7B0FED7000CA0
:10690000FF0EE3501D6EEF0E01D0F30EE76EE72E83
:1069100087EF34F00C0E1C6EE76AE72E8DEF34F033
:0E6920001C2E8CEF34F01D2E85EF34F012008B
:02692E00036AFA
:10693000026A100EE76ED890063607360236033626
:106940000B50025C0C50035805E30B50025E0C50D8
:0A695000035A062AE72EF0D71200C2
:06695A000301646B656B94
:10696000666B676B686B696B580ED66E9E0ED76E42
:0C697000010ED56ED58EF284F28A120062
:04697C00036A080E94
:10698000E76ED890073603360C50035C02E3036EC3
:08699000072AE72EF7D71200D9
:086998001CEE00F02CEE00F0F3
:1069A000F86A0F9CF5EC33F0EFEC2EF0FDD71200F7
:1069B000FF0EE350E84E1200000000D000D000D0DF
:0669C000E82EFAD71200D8
:0669C60056322E343300AE
:0469CC0056332E30E0
:0269D000340091
:0E69D20018510151E550CD50AD508C504D5034
:0269E000305035
:0269E2000000B3
:0269E4000000B1
:0A69E60011500750F34FEA4FDA4F4B
:1069F000D04F0750C54FAC4F9F4F1150115007500B
:0E6A0000F34FEA4FDA4F784F584F534F2C4F59
:026A0E00FB513A
:106A1000F651F151EC51E751E251D651BE51AE5110
:106A2000A4519D518751725157514B5133512A51A5
:046A300000FF000063
:020000040030CA
:0100010026D8
:0100020006F7
:010003000AF2
:010005008179
:010006008178
:010008000FE8
:01000900C036
:01000A000FE6
:01000B00E014
:01000C000FE4
:01000D0040B2
:0200000400F00A
:100000000A0100010004A3000000FF0000000A0133
:10001000000104012803000A0100010A0100010790
:10002000000700FFFFFFFFFFFFFF000000000000D0
:1000300000032E000061646D696E0000000070779F
:0700400000000000000000B9
:00000001FF
